:1000000040320020BD1D000019800000A91D000025
:10001000A91D0000A91D0000A91D0000000000008E
:10002000000000000000000000000000711F000040
:10003000A91D0000000000003D1F0000A91D0000D8
:100040002521000025210000252100002521000098
:100050002521000025210000252100002521000088
:100060002521000025210000252100002521000078
:100070002521000025210000252100002521000068
:100080002521000025210000252100002521000058
:100090002521000025210000252100002521000048
:1000A0002521000025210000252100002521000038
:1000B0002521000025210000252100002521000028
:1000C0002521000025210000252100002521000018
:1000D0002521000025210000252100002521000008
:1000E00025210000252100002521000025210000F8
:1000F00025210000252100002521000025210000E8
:1001000053B94AB9002908BF00281CBF4FF0FF317E
:100110004FF0FF3000F00CB8ADF1080C6DE904CEE3
:1001200000F010F8DDF804E0DDE9022304B07047C8
:10013000704700BF034613F8012B002AFBD1181AA1
:10014000013870472DE9F04786468C460846089EE0
:10015000154674461946002B40F0C2808542B2FA1B
:1001600082F245D94AB1C2F1200300FA02FC2EFA0C
:1001700003F3954043EA0C0C94404FEA154EA8B2A5
:10018000BCFBFEF8230C0EFB18CC08FB00F943EA7D
:100190000C43994528D9EB1808F1FF3704D299454B
:1001A00002D9A8F102072B44A3EB0903A4B2B3FBC5
:1001B000FEFC0EFB1C330CFB00F044EA0344A0429F
:1001C00014D92C190CF1FF3304D2A04202D9ACF19E
:1001D00002032C44241A43EA07401EB1D4400023F2
:1001E00034607360BDE8F0874746DDE76346F1E7BA
:1001F00092BB431B01214FEA154EAFB2B3FBFEFC8D
:10020000200C0EFB1C330CFB07F840EA0343984517
:1002100062D9EB180CF1FF3004D2984502D9ACF149
:1002200002002B44A3EB0803A4B2B3FBFEFC0EFBBD
:100230001C330CFB07F744EA0344A7424ED92C19A0
:100240000CF1FF3304D2A74202D9ACF102032C44D3
:10025000E41B43EA0040C0E7C2F1200320FA03F1A7
:10026000954090402EFA03F303434FEA154EAFB288
:10027000B1FBFEFC0EFB1C10190C0CFB07F841EA4D
:100280000041884504FA02F422D969180CF1FF30C4
:1002900004D2884502D9ACF102002944A1EB08013F
:1002A0009BB2B1FBFEFC0EFB1C110CFB07F743EAF3
:1002B00001439F420ED9EB180CF1FF3104D29F424B
:1002C00002D9ACF102012B44DB1B41EA004192E769
:1002D0006046E3E76146F7E76046A3E76346B7E7B2
:1002E000834206D916B9002108467BE7C6E900E03B
:1002F000F9E7B3FA83F78FB9834201D3724508D87F
:10030000BEEB020460EB030301209C461EB90021F2
:1003100068E73846FAE7C6E9004CF8E7C7F1200C71
:10032000BB4022FA0CF41C432EFA0CF120FA0CF319
:10033000B84001434FEA14490EFA07F5B3FBF9F848
:100340001FFA84FE09FB18300B0C08FB0EFA43EA77
:1003500000439A4502FA07F240D9E31808F1FF304A
:1003600004D29A4502D9A8F102002344A3EB0A0360
:1003700089B2B3FBF9F809FB183308FB0EFE41EA1A
:1003800003418E452CD9611808F1FF3304D28E4504
:1003900002D9A8F10203214443EA0040A0FB0298DD
:1003A000A1EB0E014145CE46434602D306D14D4551
:1003B00004D2B9EB020E68EB04030138002EA6D07C
:1003C000B5EB0E0261EB030101FA0CFC22FA07F314
:1003D0004CEA0303F940C6E9003198E74046C5E717
:1003E0004346D9E7F8B5174D284608F0D3F9044637
:1003F00028B32A69A968136843F0400313600B68A7
:10040000114A062128469847002818DB0F4F104E46
:10041000AB6840215B692846984700280FDB84F0D1
:10042000010414F0FF0414BF39463146094806F0B0
:100430000BFE00214FF4004006F096F9E8E700209B
:10044000F8BD00BF3090000001000600609400007D
:100450006394000067940000014B1B68184700BFBD
:10046000B0000020014B1860704700BFB0000020B2
:1004700030B585B004460D4610220021684608F0CC
:1004800006FD02238DF802302A46044B01932146D3
:10049000684606F0EBFD05B030BD00BF5904000012
:1004A00080B505460E461746984606F099F903466C
:1004B00008F058FDDFF81890044649F8003042462D
:1004C00030463946A84754F8090001F0E5FC00BF62
:1004D000080000002DE9F047058B044628079046E8
:1004E00011D4022905F0070540F0CC80204607F022
:1004F000F1FA78B10138218B042811D8DFE800F037
:10050000C2106D85950001290CBF45F0100545F01E
:100510002005258388F31188BFF36F8FBDE8F0872E
:1005200001F0070AAA4500F0A5800027B9463E461B
:10053000A368002B00F0BC8041F00801218388F300
:100540001188BFF36F8FA168002900F0BA800D6891
:10055000002900F0B680D1F8048033465246204688
:10056000C047002D76D02B6829461D46F0E701F0E4
:1005700007035A1F012A1BD8002221F00701062B6E
:10058000276889B2C4E9002209D13B4603E0628BA7
:10059000013262831B68002BF9D141F002012183F3
:1005A000204607F097FA00287AD041F0200176E043
:1005B000042B0AD121F0070189B22183204607F0DC
:1005C00089FA10B141F020012183218B01F0070A43
:1005D000AA454FD00027B946AAE7236921F00701B1
:1005E00041F00601062DD3F8009021832DD1B9F1F9
:1005F000000F3FD041F00801218388F31188BFF339
:100600006F8F3A492046C84729E021F00701236946
:1006100041F0040189B2042DD3F804902183E6D07F
:1006200000273E464FF0040A82E721F007012369C4
:1006300041F0050189B2052DD3F808902183D6D069
:1006400000273E464FF0050A72E700273E464FF06E
:10065000060A6DE72B4687E7B9F1000FD1D1EFF31A
:100660001188202383F31288BFF36F8F238B23F02D
:1006700008032383258BEA062ED525F01003238358
:1006800005F007056669218B002EBFF670AF0023C9
:100690002768C4E9003321F0070141F001012183FB
:1006A000218B01F0070AAA454FF000097FF440AF03
:1006B000002F9CD041F00801218388F31188BFF3FB
:1006C0006F8F002FC8D03D683946334652462046CA
:1006D00007F02CFA2F46F4E7AB067FF51BAF25F0A9
:1006E0002003238305F0070500E700BF597B0000C6
:1006F000014B03600020704708920000F0B40C4BDF
:100700000C4E5F6A0C4BB34203D36FF08500F0BC14
:1007100070475D68BD4209D31C693CB195F802C0C1
:100720000579AC4502D12346F0BC18472433EAE7EB
:1007300068070020C4030020A00300202DE9F04733
:10074000134CDFF85080DFF8509005460E461746F0
:10075000444503D36FF08500BDE8F0876268D9F89F
:1007600024309A4212D3A36983B1907829798842C0
:1007700005D13A4631462846BDE8F0471847527938
:10078000012A03D13A463146284698472434DFE708
:10079000A0030020C4030020680700202DE9F041D9
:1007A0000B4CDFF8308005460E461746444502D311
:1007B0006FF0850009E063690BB92434F6E73A4627
:1007C0003146284698470028F7D1BDE8F08100BFA0
:1007D000A0030020C403002010B5044607F08BFCE2
:1007E00010F1780F00D050B9054A204607F031FBD0
:1007F000D2F8C43023EA0003C2F8C430002010BD90
:1008000068070020024B00221A605A60704700BF40
:100810002308002070B50B4B0B4CA34201D30020E2
:1008200070BD196A1E7F00220439D5B2AE4201D8CC
:100830002433F2E7013211F832508542F5D101201C
:10084000EEE700BFA0030020C403002008B509485C
:100850000378C3F341130A3350F823303BB100F15E
:10086000080200F110019847C043C00F08BD1846A8
:10087000FCE700BF6807002004282DE9F14FDFF8EE
:10088000989004460F4616D001282DD1DFF88C80B1
:1008900098F8B93043B300F0D7FD214D4D4520D233
:1008A000D5F820B04FF0000A2B7F5FFA8AF6B342EA
:1008B00004D82435F2E7FFF7A5FFE7E70BEBC60600
:1008C0000AF1010A307907F016FC0246307907F088
:1008D000C0FAD8F8C430002A23EA0003C8F8C430AC
:1008E000E2DA002388F8B9300D4D4D4508D30B4BA3
:1008F0001B6A6BB13946204601B0BDE8F04F18477E
:10090000EB681BB13A462146284698472435ECE768
:1009100001B0BDE8F08F00BFC403002068070020CD
:10092000A003002073B5C4B263060D468DF80740DE
:1009300007D02046FFF76EFF78B10D4B93F8BA0051
:1009400058B10B4E204655B102F0BAF9F3691BB10C
:100950000DF1070108209847012002B070BD02F098
:10096000D7F9F369002BF7D00DF107010920F2E761
:100970006807002073B586788DF8006003794279A6
:100980001C4C43EA0223ADF80230C378304603F032
:1009900003038DF8043007F05CFAD4F8C430184231
:1009A00005460BD0304600F031FD3046FFF714FF0E
:1009B00008F076F810B9962005F0F4FE684602F0CB
:1009C0005BF910F1780F03D010B1002002B070BDB8
:1009D0009DF8000002F0D8F910F1780F01D000283E
:1009E000F3D1D4F8C43001202B4384F8B900C4F803
:1009F000C430EBE7680700202DE9F047924DAB6962
:100A000004460E461746C3B9207800F01F0001289F
:100A100076D0022800F0DC8000BB94F900103A6820
:100A2000637800292EDA062B0CD0082B25D0ABB921
:100A3000537001231370022303E198470028E3D188
:100A400000200DE06388190A0A1F012A8C4605D987
:100A5000072903D8DAB26B6A1C781CB96FF015004D
:100A6000BDE8F0875D78654503D1824200F0E480FF
:100A700001302344F0E71B78E3E095F8BA301370B7
:100A80000123DEE0052B11D0092BE7D163886E6AC4
:100A9000002B32D1FFF7B6FE638885F8BA30EB69D8
:100AA000002BCDD0694903209847C9E7A07802F010
:100AB000D1F80028C4D0D1E77378042B10D0052BCF
:100AC00011D0022B04D177796388BB4208BF012083
:100AD00033781E443378002BEED10028BED0D9E7FE
:100AE00096F80380F4E76388BB42F1D1B8F1000FB8
:100AF000EED13046FFF73EFFEAE7FF27B846E9E7C9
:100B000095F8BA30D7F800C0002BA7D06F6AA2883A
:100B100094F804E03B46187800289FD059780229C1
:100B200004D193F80480F04500F292800344F2E788
:100B30008CF800308CF80130316081E71F4493E07D
:100B40000B2B8BD100264FF0FF08C146B24606E0C2
:100B50007B78042B0FD0052B21D03B781F443B78AA
:100B6000002BF5D1EB6913B1514607209847002EB1
:100B70007FF466AF72E797F80280A38897F8039036
:100B80009845EAD163889945E7D1B8F1070F1CD899
:100B900005EB0803BA4683F8BB900126DDE7A3887E
:100BA0004345DAD1A3784B450AD0BE78304600F0F1
:100BB0002DFC3046FFF710FEB0FA80F67609CCE740
:100BC0003846FFF7D7FE0646C7E7BA460026C4E711
:100BD00094F900206378002A18DA002B7FF43EAFE6
:100BE00024793F6863060AD02046FFF713FE0028E9
:100BF0003FF434AF95F8BA30002B3FF42FAF3946AD
:100C0000204602F0A5F800237B7014E7012B08D0E2
:100C1000032B7FF423AF6388002B7FF41FAF0121E8
:100C200003E0618800297FF419AFA088FFF77AFEFE
:100C300000287FF405AF11E702293B607FF41BAF6A
:100C40005B883360FCE600BF6807002022080020B4
:100C500094F9000063780028BFF672AF002B3FF4D0
:100C600067AF0A2B7FF4FAAE3B78002B3FF4F6AE69
:100C7000797804297FF462AFB9788A427FF45EAF55
:100C8000072A96BF5219002392F8BB308CF8003027
:100C9000F6E600BF13B5164C237DF3B9E268A168F0
:100CA000019201AB802007F0E2F8019AA368134497
:100CB000A360E3689B1AE3606BB962B12369E288C1
:100CC0009A4208DD94F8C82093FBF2F102FB11333D
:100CD0000BB90123237502B010BD00231A46194633
:100CE0008020237502B0BDE8104002F077B800BF45
:100CF0006807002030B585B0002302460D460193F9
:100D0000002858D1002935D108220B460DEB0201ED
:100D100007F00AFA002804DA802001F0D1FF05B0BC
:100D200030BD2A4C029A2260039A626004F13802B4
:100D3000A2609DF90820BDF80E302575002AC4E98F
:100D400003550ADB802B04D9802001F0B9FF002075
:100D5000E3E713B1C4E90333E1E7FFF777FD0028C8
:100D6000DAD0E28823699A42D4BFE260E360FFF7F9
:100D700091FFD4E7154CD4E90215002D01AB04DC3A
:100D800007F0D2F90028CADAC6E72A4607F0CCF9FC
:100D90000028D9DB019AA3681344A360E3689B1A77
:100DA000E360002BBBD104F13803A360FFF74EFDD5
:100DB0000028DCD1B0E78028B1D1044BDA68002AE2
:100DC000D5D11B7D002BD2D1A9E700BF6807002039
:100DD000054B064A9A62064ADA62064A1A63064ACE
:100DE00058629A610020704768070020F9090000E6
:100DF000FD0600009D0700003D0700002DE9F341BE
:100E00000446474D47484FF0FF334FF0FF3204F0A0
:100E10001BFF95F8B830002B7BD16B6A83B1424839
:100E20002C62E8616E6A02F0F3F801F0E1FE041E44
:100E300010DA3C4804F080FF204602B0BDE8F081A3
:100E400000F0BEF8FFF7C4FF6B6A002BE7D14FF04C
:100E5000FF34EEE700F01AFB041EEADB7378012B87
:100E60005AD1F379002B57D00026684685F8C83050
:100E7000ADF802308DF804608DF8006001F0FCFEE2
:100E8000041ED6DB802768468DF8007001F0F4FE62
:100E9000041ECEDB2549304602F0A6F8041EC8DB4E
:100EA0002249384602F0A0F8041EC2DB204CDFF8CD
:100EB000848044451AD3002001F066FF041EB8DB8D
:100EC000D5F8C430802043F00103C5F8C43001F0E8
:100ED0005BFF041EADDBD5F8C43043F48033C5F8A6
:100EE000C430012385F8B8300024A2E7276A002621
:100EF000227FF3B29A4201D82434DAE707EBC30227
:100F000057F83310107902F06FF801360028EFD04F
:100F10009DE76FF077048CE76FF0150489E700BF59
:100F200068070020C802002079080000F50C0000C6
:100F3000A0030020C403002030B51F4B8BB005AACE
:100F400003F1100518685968144603C40833AB420E
:100F50002246F7D11B7823701022002101A807F048
:100F600096FF12220021154807F091FF102101A8D9
:100F700007F0DDF900281BDD0828B8BF0820093874
:100F800001AB0E491A18002012F8013F0AAC04EB1D
:100F9000131403F00F0328336B44013014F8144C7E
:100FA00013F8143C0C7008284B7001F10201EBD1CE
:100FB00002480BB030BD00BF76940000B51B002086
:100FC0002DE9F04F724B93F800B087B0BBF1000FE2
:100FD00003D0704807B0BDE8F08F6E4C00264FF08C
:100FE000011AB0463546B14623783BB96A4B023404
:100FF0009C42F3D1664A01231370EAE76378052B1C
:101000001BD8DFE803F08E03C38E1D39402304A8EC
:101010008DF810B0ADF812308DF814B007F056F816
:1010200040B1082304A8ADF8123007F04FF808B11A
:10103000ADF812B0BDF81230E37123781C44D3E749
:10104000E378002BF9D1A3786BB108F101085FFABE
:1010500088F8F2E76B689C4207D024354F4B9D42DD
:10106000F8D30020B6E74E4DF8E7AB68002BECD084
:10107000414620469847E8E7002DF2D000222B7F1A
:101080009A42EED2296AA07801EBC2010B7998420C
:1010900001D00132F3E70127E07800F003008DF87A
:1010A0001400207994F805C040EA0C20ADF8120035
:1010B00094F902000028FBB228DA07F110004FF083
:1010C000010C0CFA00F010EA0A0F26D143F0800060
:1010D0008DF8100004A8CDE90213019206F0F6FF86
:1010E000DDE90121039BC0B99DF81020A27012F028
:1010F000800F18BF10330A7118BFDBB24FF0010226
:1011000014BF9A40BA404AEA020A96E70120B84062
:1011100010EA0A0F01D11846DAE70137102FBBD1C8
:10112000B7E7032E1AD1FFF707FF074650B1FFF7C5
:1011300001F8024630B11028A8BF10223946A01C81
:1011400007F097FE23786FF00201E218091B04EB09
:101150005303D14213D50136F6B26EE7002EF1D11A
:10116000B9F1000F3FF47DAFA4EB090389F8023019
:10117000C3F3072389F8033089F80480EBE702F80A
:1011800001BC13F8010902F8020DE2E7A14654E799
:10119000B41B0020FC0200209F030020C403002099
:1011A000A003002010B5094B00211A461C78844288
:1011B00004D15C6814B102EB811010BD0131042927
:1011C00003F14003F2D10020F7E700BF340800200C
:1011D0002DE9F34150F8283C10F82C6C10330446EC
:1011E0000AD1036950F8202C980736D5D2B959078F
:1011F00015D5002344F8283C54F8283C10330BD074
:1012000054E9077554F8148C07F04AFC00284FD0B5
:101210002E48214607F028FC02B0BDE8F08143F0DB
:101220000403236154F8241C01AB304606F01FFE72
:1012300010B16FF01503DDE7019A54F8243C134414
:1012400044F8243C54F8203C9B1A44F8203C54F8C1
:101250001C3C134444F81C3CCEE754F8241C01AB5E
:10126000304601F037FE0028E3D1019D54F8243CBC
:101270002B4444F8243C54F8203C5B1B44F8203CAD
:1012800054F81C3C2B4444F81C3C002DB1D0304693
:1012900001F0C4FEB5FBF0F303FB1055002DA8D1FF
:1012A00054F8203C002BA4D0304601F05BFEA3E7AD
:1012B00044F8180CA4F1100004F0ACFD002DABD0E4
:1012C000424639463046A847A6E700BFC80300207B
:1012D0004B1E012B73B506460D460FD8FFF762FF74
:1012E000044668B9012D09D101AB01220DF10301BA
:1012F000304601F0EFFD019B002BF5D102B070BD2F
:1013000007F0CEFB04F12C0108B1012D05D10846F0
:1013100002B0BDE87040FFF75BBF034802B0BDE814
:10132000704007F0A1BB00BFC80300202DE9F74FB4
:10133000064601911546984606F0E4FD044600284D
:101340005BD1EFF3118A202383F31288BFF36F8FF1
:10135000DFF8ACB000220023584604F07FFD70B9DE
:10136000DFF8A090A70109EB8414636813F1100F54
:1013700014D10193584604F04DFD019B06E0013461
:10138000042C0BF1400BE5D16FF00B038AF31188AD
:10139000BFF36F8F184603B0BDE8F08F019B20614B
:1013A000C4E902350C9B63610D9BA36130466FF06D
:1013B0000F0309F80760C4F83C80636001F02EFE5B
:1013C00058B1304601F02AFEB5FBF0F303FB10558F
:1013D0001DB1E36B43F00403E36318F0020F07D081
:1013E00007F12C010848494407F03EFB0023CDE7F4
:1013F000304601F0B7FD0346C8E76FF00F03C9E7B9
:101400005008002034080020C803002010B5EFF376
:101410001184202383F31288BFF36F8FFFF7C2FE7E
:1014200050B14368103307D16FF08B03436000F174
:101430002C01044807F018FB84F31188BFF36F8F69
:1014400010BD00BFC8030020F8B50E4C04252027AE
:10145000EFF3118687F31288BFF36F8F6368103341
:1014600007D16FF08B030848636004F12C0107F08B
:10147000FBFA86F31188BFF36F8F013D04F140043E
:10148000E6D1F8BD34080020C803002070B50A4C2E
:101490000A4E00253146204607F0CAFA0122A4F17F
:1014A00010001146013507F087FA042D04F14004BD
:1014B000F0D1002070BD00BF60080020D1110000F5
:1014C00070B504460E4601791548154606F0F6FC3F
:1014D00010B394F900206378002A16DB202B04D087
:1014E000222B0ED06FF085000AE02B681A6840F8B6
:1014F000102C9A8820F80C2C9B7900F80A3C0020CC
:1015000070BD638800F8093CF9E7212BEAD1103857
:10151000072328603360F2E76FF01200F0E700BFA6
:101520003409002008B50146034806F0D5FC10B187
:10153000012300F8073C08BD34090020016901239C
:1015400081F84B300B6833B191F849301BB1024838
:10155000083107F089BA7047C803002001690123E8
:1015600081F84A300B6833B191F848301BB102481A
:10157000083107F079BA7047C803002070B501231D
:1015800082F8483013680D4614463BB192F84A3051
:1015900023B10E4802F1080107F066FAD4F8903042
:1015A0001A699B689A4205D17DB904F1180140F689
:1015B000CD4204E004F11801002DF8D00022BDE86E
:1015C00070400248002304F0A9BD70BDC80300208C
:1015D00070B5056995F89E00E0B195F89F30D3B9D4
:1015E00085F84830EFF31186202383F31288BFF388
:1015F0006F8FD5F8900006F0B7FB044686F311888C
:10160000BFF36F8F05480022002305F1180104F095
:1016100085FD204670BD0020FCE700BFC803002008
:101620000D4A03460021A0F848101068C3F8940042
:1016300090889279A3F8980083F89A2083F89C10F8
:1016400083F89B10A3F89E1083F8A010402203F1AA
:101650004C0007F01CBC00BFF8910000F0B5D0F8BA
:101660008C305B681B6A1F7D85B00446384606F0E7
:1016700049FC0646F8B994F88630E3B1A06F4FF400
:10168000806203A906F08FFB0546A0B18306A4F192
:10169000180308BF00F1FF3584F830600193074B51
:1016A000039900932A4602233846FFF73FFEA06FB6
:1016B000294606F098FB05B0F0BD00BF7D1500007F
:1016C00010B504690023C4F8A8300C4BC4F8A4007A
:1016D000596804F1A80269B9C3E9002204F10800BD
:1016E000074907F0A5F904F11800064907F0CCF9FD
:1016F000002010BD0A605A60F0E700BF34090020E6
:101700002F7F00005D16000073B504698DF8071087
:10171000002384F848302025EFF3118685F31288E2
:10172000BFF36F8F0122D4F890000DF1070106F08E
:101730001BFB86F31188BFF36F8F01280AD007F0D7
:10174000AFF910B994F8A1306BB9094B1A780AB9FE
:1017500001221A702122002304F11801054804F027
:10176000DDFC02B070BD0021212004F0FDFFD3E7B5
:10177000C71B0020C803002037B514460A1E0546C3
:1017800020DDD4F88C0004F14C0106F0EDFA0123C1
:1017900084F8493023683BB194F84B3023B11148A9
:1017A00004F1080107F060F9D4F88C104B684A691D
:1017B0009A1ACB699B1A3F2B04D8012384F8A030D6
:1017C00003B030BD94F89E30002BF9D0064B009347
:1017D00001940123402204F14C012846FFF7A6FDA5
:1017E000EEE700BFC803002079170000F7B50D46EB
:1017F00001461D4806F056FB044610B30646691E16
:1018000056F8A4395F6805291BD8DFE801F01C1AD7
:10181000031C222610F8061C99B9012300F8063C87
:101820003B6A3246187BFFF7A7FF14F85C2C42B9DD
:101830003B6A187D0D4B0093019602231146FFF77A
:1018400075FD03B0F0BD304603B0BDE8F040FFF7D2
:10185000E7BE012304F8053CF3E710F8053C002B34
:10186000EFD00023F6E700BF340900207D1500000B
:1018700037B5094D0949002400944FF0FF334FF468
:101880008062284604F00CFC0549284607F00EF952
:10189000204603B030BD00BFC8030020001C00205C
:1018A0009494000008B5044806F0ECF8BDE8084040
:1018B000024806F0E7B800BF9D940000D2940000F3
:1018C000014805F019BA00BF4C92000038B5044633
:1018D00018B90F4B0F485B6898476168B1F5683FCE
:1018E00010D0B1F5680F0DD00B4DA9420AD011F4FC
:1018F0006861206807D00146084806F0A6FF00236B
:101900002360656038BD142207F0C1FAF9E700BF13
:10191000F0010020009500002C5F5CA93C0E002027
:1019200008B520B34368B3F5683F10D101220368BE
:10193000BFF35B8F53E8001F002903D143E8002069
:101940000028F7D1BFF35B8F0DD1002008BD094AF5
:1019500093420AD000684FF0FF324FF0FF3304F09B
:1019600073F90028F1D00448F0E70448EEE76FF47B
:10197000E040EBE72C5F5CA9E98FFFFFEA8FFFFFF8
:1019800008B5D8B14368B3F5683F10D100220368A9
:10199000BFF35B8F53E8001F012903D143E8002008
:1019A0000028F7D1BFF35B8F0BD1002008BD074A99
:1019B000934208D0006804F0BFF9F6E76FF4E04006
:1019C000F4E70348F2E70348F0E700BF2C5F5CA9A7
:1019D000E98FFFFFEA8FFFFF10B5044618B91D4BD2
:1019E0001D485B6898476368B3F5683F2FD0B3F52F
:1019F000680F2CD0194A934219D1236803BB1848A9
:101A00004FF0FF324FF0FF33214604F0EFF808B9F2
:101A100023681BB90F4B13485B6898472068142252
:101A2000002107F034FA4FF46863636008E0B3F50F
:101A3000683F0DD83A2B03D040F6BA629342DED10C
:101A4000206806F03AFF636843F03A03636010BD14
:101A5000054AF3E7F0010020009500002C5F5CA927
:101A60003C0E0020269500003A00003A08B50649D1
:101A700006484023142206F0DAFEBDE80840044977
:101A8000044805F0ABB900BF3C0900203C0E002023
:101A9000549200006892000030BFFFF7FDBF00BF06
:101AA0002DE9F0410B4EDFF8308006EB0807CC1B28
:101AB000054632460949204607F0DBF9A01942469F
:101AC0000021083C07F0E3F92C6707F10800BDE8A6
:101AD000F08100BF0000000004000000EC91000055
:101AE000074A936893F90E10002907DB5269934265
:101AF0001FBF044A536843F080535360704700BFD0
:101B0000A419002000ED00E070B5264B15469A6A36
:101B100012F0100F9A6A14BF1124102412F0080F4B
:101B20009A6A18BF1224920706460AD5586B9A6A19
:101B3000140634D519B19A6A22F080029A621324ED
:101B400001E06FF01500174B9A6A12F0010F9A6AC4
:101B500018BF142412F0200F9A6A18BF1524D20659
:101B600002D49B6A9B070AD50E4B5B68190506D504
:101B7000314600F08DFA10B180F309880224094B38
:101B80009A6A920642BF5A6A22F400525A629A6ACC
:101B900042F0FF029A6200232B70204670BD6FF066
:101BA0001500CCE700ED00E0134B9A6A12F0007FBD
:101BB0009A6A14BF1E201D2012F0807F9A6A18BFF7
:101BC0001F2012F4002F9A6A18BF212012F4802FD0
:101BD0009A6A18BF222012F4003F9A6A18BF232085
:101BE00012F4803F9A6A6FEA02426FEA12429A62E6
:101BF00018BF2420704700BF00ED00E010B5194B5E
:101C00000246986A9C6A10F4805F14BF1720162061
:101C100014F4006F9C6A18BF1820A40509D5986BAE
:101C2000986A000404D51AB19A6A22F400429A62B2
:101C300019200C4B9A6A12F4806F9A6A18BF1A2006
:101C4000D2050CD49B6A13F4005F18BF1C20054A10
:101C5000936A43F47F43936200230B7010BD1B20F3
:101C6000F5E700BF00ED00E0F0B5484B5B688BB0D6
:101C70000446C3F30803002585F31188BFF36F8F73
:101C800002F07F40B0F17F4F11D102F00C00082824
:101C90000DD010074CBF0C4601250022033B8DF8E8
:101CA0000720032B05D8DFE803F0246367602C4688
:101CB000F3E700239DF80720CAB902AE04F120071C
:101CC00020686168324603C20834BC421646F7D128
:101CD000099A002D54D0C2F3080121B96FEA5222AB
:101CE0006FEA4222099202A9184606F08BF90BB05E
:101CF000F0BD264BDA6A9107DBD4DA6A002AD8DB1A
:101D0000DA6A5200D5D55A69A16942F480725A61E3
:101D1000BFF34F8FBFF36F8F5A6931F8021C22F463
:101D200080725A61BFF34F8FBFF36F8F4DF602720F
:101D300091420AD09A6AD2B24AB10DF1070201214A
:101D40002046FFF7E1FE0346B4E72368B2E79A6A4C
:101D500012F47F4F05D00DF107010120FFF74EFF70
:101D6000F1E79B6AB3F5803FA3D3FFF71DFFEAE7D6
:101D70000DF107020021E3E70DF107010020EDE777
:101D800022F4FF7222F00102ACE700BF00ED00E098
:101D9000044B5A6942F010025A615A6922F0080253
:101DA0005A61704700ED00E0EFF30880EFF309811E
:101DB00001B57246FFF758FF01BD00BF002080F358
:101DC0001488BFF36F8F02F0E7FE00200D49086012
:101DD000BFF34F8F0C4880F3088800F02BF82020C9
:101DE00080F3118809484FF40461401880F3098892
:101DF000EFF314800221084380F31488BFF36F8F40
:101E000000F00EF994ED00E0403200208024002024
:101E10000749D1F890200023C2F3072218469342C5
:101E200000DB7047C1F89830C1F8A0000133F6E735
:101E300000ED00E008B572B6002383F31388FFF7C6
:101E4000E7FF144B4FF0FF32C3F88020C3F8842023
:101E5000C3F88820C3F88C20C3F89020C3F89420DE
:101E6000C3F89820C3F89C20C3F88021C3F88421CC
:101E7000C3F88821C3F88C21C3F89021C3F89421BA
:101E8000C3F89821C3F89C2162B6BFF34F8FBFF30C
:101E90006F8F08BD00E100E0084B9B6883420BD1C7
:101EA000EFF3058343B1064B5A6842F080525A6003
:101EB0005A6A22F400425A6206F0CDBEA4190020EC
:101EC00000ED00E0094A93686FF00A01996708493C
:101ED00058674B6843F080534B60002383F31188AD
:101EE000BFF36F8F9368986F704700BFA4190020ED
:101EF00000ED00E010B50446EFF31183202383F3D7
:101F00001288BFF36F8F0A4B58699860094B4FF0E6
:101F100000625A60084B026F1A600022436F4267EA
:101F200083F31188BFF36F8F00F01AF9204610BDBC
:101F3000A419002000ED00E0580E00200B498A682B
:101F40004FF030001044EFF3098C80E8F01F744626
:101F50007046FFF7CFFFA64604498A6802F13000B9
:101F600090E8F01F8CF3098870470000A419002046
:101F70001EF0040F0CBFEFF30880EFF309808169B6
:101F800011F8021C0229FFD001B506F041F801BD8D
:101F900040B2002807DB044A4109012300F01F007A
:101FA000834042F82130704700E100E040B2002851
:101FB0000CDB4309064900F01F0020330122824058
:101FC00041F82320BFF34F8FBFF36F8F704700BFDF
:101FD00000E100E0054B420900F01F0053F8222009
:101FE000012303FA00F01040704700BF00E100E059
:101FF00040B20028A8BF00F1604001F10101B8BF64
:10200000064B4FEA4111ACBF00F5614000F00F00F4
:10201000C9B2B4BF195480F80013704714ED00E042
:102020000B4A08B50B4B22F07F029A60BFF34F8F2B
:10203000BFF36F8FD3F8882022F47002C3F8882092
:1020400003F010FD04F06AFC00F060F803F04EFDB0
:102050000000000000ED00E042F8203C009B42F848
:102060001C3C0A49019B42F8183C029B42F8143C74
:1020700021F001014FF0807342F8043C42F8081C43
:102080000023203A02654367704700BFA1040000A7
:10209000094A0346906870B113F1160F006E05D01F
:1020A000A0F140029A4205D8834203D2814228BF60
:1020B0000020704700207047A419002008B515467D
:1020C0000B4A0C4B9060026F1A600E4600F048F805
:1020D0002C4686F309884FF00000074B98472046AE
:1020E0004FF000014FF000024FF00003034C204777
:1020F000A4190020580E00202F800000A104000029
:10210000014B10221A61704700ED00E004480023E3
:102110002021C2180133302B82F80013F9D1704707
:1021200000E100E008B5EFF30583064A103B02EB3F
:10213000C30152F8330049688847BDE80840FFF7FB
:10214000CFBC00BF6C900000024B034A0348012142
:1021500000F076B800000420000000207892000013
:10216000026E054B403A1A60044A4021C3E901124D
:102170001846012100F06EB85C0E002000000B151F
:10218000084AC2F898000B6823F01F03034343F08A
:102190001003C2F89C308B6843F00103C2F8A030F2
:1021A000704700BF00ED00E02DE9F043DFF86080EC
:1021B00085B00E461F4604464FF00009B14523DAAC
:1021C0006068D8B13FB1411E08421BD11F2819D900
:1021D0002368194216D12368019305F04BFFA368C9
:1021E00003430393D8F89050C5F30725D0B2013DBF
:1021F000A84207D801A9FFF7C3FF421C09F1010952
:102200000C34DBE76FF01502104605B0BDE8F08333
:1022100000ED00E0044B0522C3F89420BFF34F8F7C
:10222000BFF36F8F704700BF00ED00E0BFF35F8F1B
:10223000024B0022C3F89420704700BF00ED00E07D
:1022400010B5034C01232278FFF7AEFF207010BDBC
:10225000C81B002008B50B4A00231278FFF7A4FF23
:1022600010F1160F07D0084A0021D2F89030C3F3BE
:102270000723984200DB08BDC2F89800C2F8A010FE
:102280000130F2E7C81B002000ED00E02DE9F0432B
:10229000534B544CD3F890302568C3F307239D4229
:1022A00085B000F29A80FFF7C1FF00200C2685421E
:1022B0001AD14D4C4D4F25706846FEF719FADFF8DC
:1022C0002081DFF82C9106460025AE4213D12378F9
:1022D00043490020D1F89020C2F30722934276DBD5
:1022E000FFF798FF002042E0616806FB0011FFF74E
:1022F00047FF0130DBE7009800EB05114FEA051CB2
:10230000CB683B40B3F5000F48D00AD8B3F5001FA7
:1023100030D0B3F5800F36D0B3F5801F10D0013523
:10232000D3E7B3F1807F42D0B3F1007FF7D150F80B
:102330000C3088684A6805F09DFE40F4802009E072
:1023400050F80C3088684A6805F094FE40F08850D8
:1023500040F43020CDE901230390D8F89030207864
:10236000C3F30723013B98422AD96FF0150005B04B
:10237000BDE8F08350F80C3088684A6805F07AFEB2
:1023800040EA0900E6E750F80C3088684A6805F032
:1023900071FE40F0E06040F40030DBE750F80C30B4
:1023A00088684A6805F066FE40F08270D2E750F80F
:1023B0000C3088684A6805F05DFE40F08870C9E717
:1023C00001A9FFF7DDFE237801332370A7E7C1F8E9
:1023D0009830C1F8A00001337CE74FF0FF30C6E72A
:1023E00000ED00E084920000C81B00200000F0FF18
:1023F0000000081108B5024B1B689847002008BD73
:10240000680E0020034B044A1860937843F00203DF
:1024100093707047680E00202C01002008B5064913
:10242000064821F00701C1F1005202F5802205F0B3
:10243000CFFA002008BD00BF474100206C0E0020ED
:102440000E4A0123C2F840354FF080424FF08051D0
:10245000C2F87835D1F83001082808D1D1F8341104
:10246000052904D80648415C09B1C2F838364FF056
:1024700080430122C3F880250020704700E001401E
:102480006295000020B1034B800143F0010318471F
:10249000704700BF009200004FF08043D3F84036F1
:1024A000DB072ED54FF01023D3F8043303F00703D6
:1024B000072B26D1144A0123C2F80435D2F8003480
:1024C000002BFBD04FF01021D1F8043323F0070389
:1024D00043F00403C1F804330023C2F804350A4A68
:1024E000D2F80034002BFBD0BFF34F8F0749084BC5
:1024F000CA6802F4E0621343CB60BFF34F8F00BFA2
:10250000FDE70020704700BF00E0014000ED00E063
:102510000400FA05020600F07F0312D5082B05D14E
:10252000010700F00F0306D50E48704710F0780F32
:1025300012D100F00F034C2000EB43100A4B18445B
:102540007047082B05D1020700F00F0306D5074896
:10255000704710F0780FF6D000207047044800EB69
:1025600043107047C40F0020780E0020E4100020B4
:10257000E40F00200149024806F076BAA00E0020C0
:10258000680400200146014806F00BBAEC02002066
:1025900002480022002303F00BBC00BFEC02002025
:1025A00013B5124800F0C4FE114B98421AD11148DD
:1025B00003F022F90024104803F064F90F49104891
:1025C00000944FF0FF334FF4806203F069FD0D4932
:1025D0000B4806F06BFA0C480C4906F029FA204625
:1025E00002B010BD6FF00400FAE700BFF52700004D
:1025F0000000AD0B76950000A8920000402000205E
:102600006804002068950000A00E00201129000039
:1026100010B50E49BFF35B8F002351E8002F012A4C
:1026200003D141E800300028F7D1BFF35B8F0CD114
:1026300051F8044C1439204605F029FB783004D1B8
:102640002046BDE8104005F0FEBA10BD980E0020EF
:1026500038B5002464F07F00C0B2FFF75BFF01349F
:1026600005F01DFD082CF5D10E4D0024E0B2FFF75A
:1026700051FF036903B90561013405F010FD082C11
:1026800005F14005F2D1084805F009FD074BD3F8E4
:102690007C2212B9064AC3F87C22064805F0FFFCEA
:1026A000002038BD08150020C40F0020780E00203F
:1026B00008110020E410002010B5054CFFF768FF5A
:1026C00020B14168204606F0C0F8F7E710BD00BF12
:1026D0005C02002007B500230E48002201A903F088
:1026E00085FA90B1FFF7E8FF0A480022002301A90C
:1026F00003F07CFA38B90198042340600374FFF7B3
:1027000041FFFFF737FF002001E00198406003B070
:102710005DF804FB5C020020022810B511D8094BBB
:102720001C5CFFF7D7FF60B1002202740472FFF750
:1027300029FF054B93F824301BB1BDE81040FFF78B
:1027400019BF10BD73950000780E0020F8B587788A
:1027500006463846FFF7DEFE3B06F578044612D5FE
:10276000002D43D1FFF7B6FF034600283ED00122DB
:10277000A5770274032202739C60FFF703FFBDE894
:10278000F840FFF7F7BE4DB1012D2FD1FFF7A2FFA3
:10279000034658B3657705740573EDE7FFF79AFFB5
:1027A00020B3B278124B12F0800F02F0080111D062
:1027B00041B1D3F8A836E360012303740223037305
:1027C0008460DAE702F00F02142101FB0233D3F830
:1027D0000836F0E711B1D3F8A837ECE702F00F02A2
:1027E000142101FB0233D3F80837E4E7F8BD00BF3A
:1027F00000700240F0B5064689B01422002103A8FB
:1028000006F045FB3378013B052B21D8DFE803F0C8
:102810007A0314146A1603238DF814300024FFF78A
:1028200059FF0346A0B1047400F10802DDE9050177
:1028300082E8030018461DE00423EDE7B778384628
:10284000FFF768FE837A044623B1013B022B43D98C
:1028500009B0F0BD3B06F57813D5002DF8D1FFF790
:1028600039FF03460028F3D00122A5770274032222
:1028700002739C60FFF786FE09B0BDE8F040FFF7E9
:1028800079BE55B1012DE3D1FFF724FF034600289F
:10289000DED0657705740573EBE7FFF71BFF07468E
:1028A0000028D5D00123037402230373846004F14C
:1028B0000C01B07805F054FC134AE168B2F88C3290
:1028C0008B4206D95B1AA2F88C3201F07FF83846A9
:1028D000D0E7A2F88C52FAE7304609B0BDE8F040E4
:1028E000FFF734BF01A801F04FF89DF80530052B24
:1028F00004D19DF8043013F0600FA9D0034B059369
:1029000001248CE702248AE7780E0020E40F0020DF
:102910002DE9F043A64CDFF89C9285B08046FFF786
:1029200037FE074610B905B0BDE8F08394F82530AE
:102930003A7C3BB9002A00F0868079689D4805F012
:1029400084FFECE7042A42D8DFE812F07D0005009E
:102950000001160140013B7BBD68032B37D8DFE83F
:1029600003F0023D5A5F6E69934B00223260726041
:10297000D3F880143170D3F884147170D3F88814AC
:10298000D3F88C0441EA00217180D3F89014D3F875
:10299000940441EA0021B180D3F89814D3F89C3410
:1029A00041EA0323F3800823EB6030687168834BAE
:1029B00003C311462B68687A984796F90030002BBC
:1029C00008DBF38833B1A4F88C3200F0FFFF79689C
:1029D0004846B4E70023A4F88C32F8E76B7F002B5D
:1029E000F5D02B7F002BF2D000266E774FF0FF3210
:1029F00073482E774FF0FF3305F064FB6B6901934A
:102A00006B68CDE9023601A9687A00F0E7FC6C48F2
:102A100005F05AFBDBE72B680121687A9847D6E777
:102A2000AB7A6BB9EB7F5BB965484FF0FF324FF083
:102A3000FF3305F047FB00F0CFFF614805F044FB92
:102A40002B680221E9E73A7A042AC0D8DFE802F0CD
:102A500059032367730000F02BFC05460028B6D10C
:102A600000F066FBBFF35B8F5649012351E8002F4E
:102A7000002A03D141E800300028F7D1BFF35B8F73
:102A8000A5D141F8085C41F8105CE0696361143934
:102A900005F082F89BE7002565F07F00C0B2FFF7E4
:102AA00039FD037A13B1407A01F0FAF80135082DA7
:102AB000F2D194F854311BB194F8550101F0F0F8BB
:102AC0000025E8B2FFF726FD037A13B1407A01F042
:102AD000E7F80135082DF4D194F874321BB194F85D
:102AE000750201F0DDF8002000F0C6FB012384F838
:102AF00025302368002B3FF46AAF0021022098475D
:102B000065E7002584F8255001F030F8FFF780FDD7
:102B10002368002B3FF45BAF29460420EFE7002B2E
:102B20003FF455AF00F0CEFB2368002B3FF44FAFCE
:102B300000210520E3E72268002A3FF448AF002B7C
:102B40003FF445AF00210620904740E708F110050B
:102B50004FF0FF334FF0FF32284605F0B3FAFFF78E
:102B600077FD284605F0B0FA58F8283C002B3FF4D2
:102B70002EAF00210120C2E794F874327BB1012509
:102B800084F8895284F88852FFF7A4FD38B10E4AC0
:102B9000057405738260FFF7F5FCFFF7EBFC58F84E
:102BA000283C002B3FF413AF00210A20A7E700BF09
:102BB000780E00205C020020007002407C0E002095
:102BC000B00E0020980E0020E410002005F0CFFD8C
:102BD00000F0CCFF00F0A2FAFFF76EFDFFF738FD22
:102BE00005F0BEFD014800F0A3FBF0E6F52700006C
:102BF00038B5164D95F824402CBB05F1380005F08A
:102C00005CFE204601F09EF922460121E861272062
:102C1000FFF7EEF905F0A4FDFFF71AFD044610B921
:102C2000012385F824300A4B1B680BB1FFF7A2FC87
:102C30004FF08043D3F83834DB0702D50020FFF78C
:102C40006BFD204638BD0024FBE700BF780E002056
:102C5000EC020020074B93F824203AB193F825307A
:102C6000002B14BF00206FF0120070476FF01200AD
:102C7000704700BF780E002038B5104B93F8243011
:102C80000446C3B105782846FFF744FC10B96FF03D
:102C9000150038BD457223798372638843602078BC
:102CA000618810F0080F02D14B1E0B42EFD105F0E6
:102CB00052FA0020EDE76FF01200EAE7780E0020EC
:102CC00038B5124B93F824200546CAB193F8253045
:102CD000B3B1FFF71FFC0446A8B1837A012B12D0D1
:102CE00007D9023B012B07D96369A3610020E0608B
:102CF00038BD00F077FEF7E7284600F019FEF3E74D
:102D00006FF01200F4E76FF01500F1E7780E002085
:102D100038B50E4B93F82420054682B193F8253040
:102D20006BB1FFF7F7FB68B115F008040AD128462C
:102D300000F020FE284600F0EBFF204638BD6FF083
:102D40001200FBE76FF01500F8E700BF780E0020D7
:102D500038B50C4B93F8242005460C4662B193F825
:102D600025304BB1FFF7D6FB48B144B1284600F0FF
:102D7000E7FD2070002038BD6FF01200FBE76FF018
:102D80001500F8E7780E002070B5134E96F8243041
:102D90000446C3B1FFF7BEFB0546B8B1230705D40F
:102DA000204600F0E7FD204600F0B2FF2B7A83B901
:102DB00001232B7296F825300BB9002070BD2046F8
:102DC00000F06EFFF9E76FF01200F7E76FF0150003
:102DD000F4E76FF07700F1E7780E00202DE9F0437B
:102DE000DFF8E4801E4698F8243085B0074689460F
:102DF0001546002B61D098F82530002B5DD00306D6
:102E00005ED5FFF787FB0446002859D0037A002BD4
:102E100056D04FF0FF334FF0FF3208F1380005F085
:102E200051F9A37F4BB108F1380005F04DF96FF06F
:102E30000A04204605B0BDE8F083A37AC5B13BB3D0
:102E40000123A3774FF0000801A93846CDE9019589
:102E5000CDF80C8000F0C2FA1C4B984229D084F8BF
:102E60001E801EBB6FF00404194805F02DF9E0E741
:102E7000E27F02B1E577002BE2D100F0B9FD874295
:102E8000DED000F0A9FD124805F01EF90024D0E7BD
:102E9000B8F80A309D42F0D26268B5FBF2F302FB4B
:102EA0001353002BE9D10123E377E6E7C6F800804E
:102EB000D8E706B135600024D6E76FF01204B8E712
:102EC0006FF01504B5E700BF780E00200000AD0BD1
:102ED000B00E00202DE9F0411D46204B174693F817
:102EE00024200E46002A33D093F8253083B30306FE
:102EF00031D401B97FBBFFF70DFB044658B3037A09
:102F00004BB34FF0FF3316484FF0FF3205F0DAF8BD
:102F1000E368BB42984628BFB84646B93FB905B1F9
:102F20002B600F4805F0D0F80020BDE8F081A169C2
:102F30004246304605F09DFFA3694344A361E36820
:102F4000A3EB0803E360002DEBD0C5F80080E8E7B1
:102F50006FF01200E9E76FF01500E6E7780E002049
:102F6000B00E002070B51E4D95F82420034682B3A4
:102F700095F825206AB31B062ED4FFF7CBFA04463A
:102F800050B3037A43B34FF0FF334FF0FF3205F1F4
:102F9000380005F097F8E368B3B90126636926772E
:102FA000A361637F83B1FFF795FB30B905F138006A
:102FB00005F08AF86FF00B0070BD0674846006732C
:102FC000FFF7E0FAFFF7D6FA064805F07DF8002093
:102FD000F2E76FF01200EFE76FF01500ECE700BFCB
:102FE000780E0020B00E002010B5084B93F8243066
:102FF0000C462BB1FFF78EFA28B10460002010BDFB
:103000006FF01200FBE76FF01500F8E7780E002074
:10301000014B1860704700BF780E002008B5074BC1
:1030200093F8243023B1FFF775FA20B1406808BD4A
:103030006FF01200FBE76FF01500F8E7780E002044
:103040004FF08053D3F83021082A06D1D3F8343119
:10305000052B04D8034AD05C70470020704701203C
:10306000704700BF77950000064B10F0800FA3F16A
:10307000D80208BF134600F00F00182202FB0030F0
:10308000704700BF20180020EFF31180202383F346
:103090001288BFF36F8F0A4BD3F8001C032261B96B
:1030A00049F27531C3F8001CC3F8142DC3F8001C95
:1030B00080F31188BFF36F8F7047C3F8142DF7E7C3
:1030C00000E00640EFF31180202383F31288BFF362
:1030D0006F8F0A4BD3F8001C61B949F27532C3F8FF
:1030E000002CC3F8141DC3F8002C80F31188BFF323
:1030F0006F8F70470022C3F8142DF6E700E00640FA
:103100004FF08053D3F83031082B02BF024B00221E
:10311000C3F81C2C704700BF00700240024A002315
:103120001360024A1370704700190020CD1B002065
:1031300008B54A4B4FF40062C3F80024FFF780FF44
:1031400008B1FFF7A1FF4FF08053D3F83031082BBF
:1031500018D1EFF31180202383F31288BFF36F8F10
:103160003F4BD3F8001CC02200296ED149F27531C3
:10317000C3F8001CC3F8142CC3F8001C80F311889A
:10318000BFF36F8F354B0122C3F80025D3F800241D
:103190001205FBD54FF40062C3F800244FF08053B2
:1031A000D3F83031082B17D1EFF31180202383F3AC
:1031B0001288BFF36F8F2A4BD3F8001C002947D128
:1031C00049F27532C3F8002CC3F8141CC3F8002C64
:1031D00080F31188BFF36F8FFFF732FF30B1FFF735
:1031E00071FFFFF72DFF08B1FFF74EFF4FF080533F
:1031F000D3F83031082B194B0AD140F2E372C3F8EF
:1032000000284022C3F80428BFF36F8FBFF34F8F0D
:103210008022C3F81C250122C3F83025114B40F24F
:10322000FF121A60104B00211960104B1970FFF744
:1032300067FF0F4B19700F4B02221A70FFF700FF48
:1032400050B1BDE80840FFF73DBFC3F8142C95E727
:103250000022C3F8142CBBE708BD00BF0070024079
:1032600000E00640FC180020F8180020C91B0020D0
:10327000CB1B0020CD1B0020094B002210B51A707B
:10328000084A094B094C002808BF1346C4F800330C
:103290002720FEF77DFE0123C4F8043510BD00BFD2
:1032A000CC1B0020FDFFDF01FDFFFF01007002408D
:1032B000034B1878012894BF00200120704700BFFD
:1032C000CD1B002010B54FF0FF324FF0FF331548F3
:1032D00002F0C4FDEFF31181202383F31288BFF3C2
:1032E0006F8F114B1B7803F0FF0483B10F4BD3F8A2
:1032F000002412F400720AD10120C3F82C05D3F87F
:103300002C05D3F80004800502D5C3F82C25002431
:1033100081F31188BFF36F8F024802F07BFD2046D6
:1033200010BD00BFDC020020CC1B0020007002405A
:10333000F8B51C4B1C7894BB1B4A106001221A7014
:1033400040F2FF17264664F07F0514F0080FEDB237
:1033500014BF39464021284604F0FDFE2846FFF7F9
:1033600083FE0134092C867506730661EBD10024B7
:1033700040F2FF17254614F0080FE6B214BF394695
:103380004021304604F0E7FE3046FFF76DFE013481
:10339000092C857505730561EDD10448F8BD044815
:1033A000FCE700BFCD1B0020001900200000AD0B82
:1033B0000500AD0B084B10F0800F00F00F0114BF9B
:1033C000D3F81025D3F8142501238B40134214BFE2
:1033D00001200020704700BF007002402DE9F84333
:1033E0000246EFF31187202383F31288BFF36F8F18
:1033F000030703D1184B1B78834229D1174B184E72
:103400001C683568104604F09EFEE443A4B24FF0F9
:1034100001092C4309FA00F814EA08041AD11046ED
:10342000FFF722FE80F80C90034607C91C6183E871
:1034300007009C750B4B0C4845EA08058022356057
:10344000C3F8042187F31188BFF36F8FBDE8F883B9
:103450000648F7E70648F5E7CB1B0020FC180020DC
:10346000F818002000E100E00000AD0B0A00AD0BF1
:103470000B00AD0B10F0080F074B06D0D3F8C004BB
:1034800010F4803F18BF0020704700F00F0000F5D7
:10349000947053F820007047007002402DE9F74FF8
:1034A000AB4BAC4ED3F85421DAB10022C3F854210F
:1034B000D3F80413890214D58DF80420D3F82025FD
:1034C000ADF80620D3F8C034002B336814BF4FF09A
:1034D00001224FF48072134333609F4B01A81B6895
:1034E00098479B4BD3F8604134B10022C3F8602168
:1034F000D3F86C44C3F86C44D3F828214AB10022B5
:10350000C3F82821954B187804F01DFE0123834051
:103510001C43DFF84C82934F98F8005098F90090C4
:1035200015F0080143D1B9F1000F05F00F032EDAB1
:103530008D4A52F8230020B342F82310142253433B
:1035400003F1804303F51C33D3F80836874A11781A
:1035500003F001034B401370FFF7D2FD844802F0E3
:1035600059FC2846FFF780FD837D032B37D1284681
:1035700004F0E9FD012303FA00F03B6823EA0003AD
:103580003B60DFF8D4A101254FF006095DE0794AE0
:1035900052F823000028F4D042F823101422534399
:1035A00003F1804303F51C33D3F80837CEE7B9F1B4
:1035B000000F674B09DBD3F85021002AE1D000222D
:1035C000C3F85021D3F8A837C0E7D3F82C21002A3C
:1035D000D7D00022C3F82C21D3F8A836B6E7037B56
:1035E000DBB9284604F0AFFD012303FA00F03B6885
:1035F000B9F1000F23EA00033B6001DA882DC0D146
:1036000006238DF8043000238DF80730524B8DF8D7
:1036100006501B6801A89847B3E7002DB1D14C4B69
:103620000122DA64ADE794FAA4F03268B0FA80F0CF
:1036300005FA00F31A430F28326024EA03043A68BB
:1036400040F39C80134200F0A980002CEBD1404B4A
:10365000D3F800215AB1C3F80041474B1C703F4BCF
:103660001C70012301933C4B01A81B689847384B01
:10367000D3F85821002A2ED00022C3F85821D3F8BD
:103680000044C3F80044E30508D53B4B01221A70FF
:1036900002230193304B01A81B689847A50508D564
:1036A000354B00221A70032301932B4B01A81B6892
:1036B000984760050FD5304B1A7862B100221A7016
:1036C000234B0122C3F808259A6504230193224B5A
:1036D00001A81B6898471E4BD3F85C3103B3244BF9
:1036E0009B681BB998F80030590619D0184B002276
:1036F000C3F85C21D3F88034184A23F07F03137099
:103700003B6823F001133B60336823F4803343F0BC
:1037100001033360052301930F4B01A81B689847F1
:103720003A6833681A4200F0EB8011480022002307
:1037300002F094FB002840F0E380054BD3F82C35D1
:10374000002B7BD00A4803B0BDE8F04F02F062BB0B
:1037500000700240FC18002000190020CB1B002044
:10376000CA1B0020F818002008710240C91B002065
:10377000DC02002030710240CC1B002013407FF49B
:1037800064AF60F07F018DF804908DF806108DF81D
:103790000730DAF8003001A8984756E7A0F1100189
:1037A0008DF804908DF806108DF80750F1E749F078
:1037B00080052846FFF758FC4368B0F814A001685C
:1037C0009A4528BF9A4601F06043B3F1005F044672
:1037D00004D05448524605F04CFB524922686368B5
:1037E00052442260A268A3EB0A03D20768B2636066
:1037F00053D5BAF1000F52D1002323734FE0114685
:103800004FF0000A604545D1003B18BF0123002A54
:1038100042D0504540D9012303FA09F32BEA0303B0
:103820003B6006238DF804303F4B8DF80650022292
:103830001B68A2758DF8072001A89847D7F800B03B
:1038400033681BEA03093FF47DAF19F0012314BF6D
:1038500093FAA3F999FAA9F9B9FA89F9B9F10F0F0D
:10386000A5D9A9F11005EDB22846FFF7FDFB0446E6
:103870002846FFF7FFFD6368B4F814C02268984239
:10388000BDD81B1A00EB020E11466360C4F800E0BD
:103890008246B7E70023BAE768B2002BACD04FF0FE
:1038A0008053D3F83031082B02BF204B8222C3F85B
:1038B0001C2C336888F80050012202FA09F923EA27
:1038C00009033360236915F0080F53442361174B34
:1038D00019D1002805F00F054FF0140000FB05304A
:1038E000A9BF0A3503EB8503C0F80017C0F804A789
:1038F000AFBF43F82520C0F80016C0F804A65A60F0
:1039000003B0BDE8F08F0028B5BFC3F8A016C3F818
:10391000A017C3F8A4A6C3F8A4A7B4BF5A629A64B8
:10392000EEE700BF081700200019002000700240D9
:10393000024B40F48070C3F81805704700700240D5
:10394000030713D400F00F0310F0800F084A0BBFD9
:1039500003F5887303F5847302EB830252F82300A6
:1039600008BF5068003818BF01207047002070471A
:1039700000700240034BC3F80C0540F48070C3F89C
:103980000C057047007002400023036043600E4B3B
:10399000D3F880240270D3F884244270D3F88824AA
:1039A000D3F88C1442EA01224280D3F89024D3F851
:1039B000941442EA01228280D3F89824D3F89C34EC
:1039C00042EA0323C380704700700240014B01228A
:1039D000DA64704700700240014B01221A6570479B
:1039E00000700240014B01225A657047007002408E
:1039F000014B1878704700BFCB1B002010B5024662
:103A0000EFF31184202383F31288BFF36F8F04F048
:103A10009AFB0B49012303FA00F00B6823EA000329
:103A20000B6012F0080101BF02F00F02054B02F516
:103A3000947243F8221084F31188BFF36F8F10BD86
:103A4000FC18002000700240F7B50146EFF3118525
:103A5000202383F31288BFF36F8FFFF705FB064621
:103A6000084604F070FB012211F0800F02FA00F208
:103A70002D4818D1036832EA03040AD00846FFF73C
:103A8000BDFF0323B37585F31188BFF36F8F03B0B8
:103A9000F0BD2649347323EA020303600B6823EA6E
:103AA00002030B60EDE70B0715D48029204B2FD0C4
:103AB00001F00F0404F2DA346400C3F80048D3F8CC
:103AC0000448D3F80478E4B244F002043C43C3F859
:103AD0000448D3F80438154F04683B6864EA030CC3
:103AE0001CEA020FCFD013433B6000233373032340
:103AF000B3758DF807300F4B8DF8061024EA0204D9
:103B0000062204601B688DF8042001A89847BAE7D4
:103B100040F2B474C3F80048D3F80448D3F80478EA
:103B2000E4B244F00404D1E7F8180020FC180020A7
:103B3000007002400019002038B50446094D4FF0CE
:103B4000FF324FF0FF33284602F088F92046FFF796
:103B50007BFF284602F05EF9034B8022C3F8042164
:103B600038BD00BFDC02002000E100E0F8B54FF0F6
:103B7000FF324FF0FF332B4802F070F92A4B8022BE
:103B8000C3F884212720FEF725FA98B1274E284B49
:103B900034681B68240C24041C43012764BB254D96
:103BA00040F2FF1333602720C5F80445FEF7FEF905
:103BB000C5F80043204A13788BB11E4B0021C3F88F
:103BC00008110121C3F80026C3F804165960D3F880
:103BD00008110029FBD00021C3F808111170154B02
:103BE0000022C3F80025FFF78BFA0E4802F012F905
:103BF000124B01221A70F8BD94FAA4F5B5FA85F5B6
:103C00000F2D2846C6BFA5F11000C0B240F08000BD
:103C1000030701D4FFF718FF07FA05F524EA0504A6
:103C2000BCE700BFDC02002000E100E0FC1800203F
:103C3000F818002000700240C91B0020CD1B002096
:103C400010B504464FF0FF324FF0FF33114802F039
:103C500005F92046FFF7F8FE04F00F020123934018
:103C60000D4A14F0800F14BFD2F81015D2F81415B5
:103C70006FEA030315BF0B400B40C2F81035C2F8C2
:103C80001435044802F0C6F8044B8022C3F804211E
:103C900010BD00BFDC0200200070024000E100E027
:103CA00070B50446FFF786FB68B904F00F020125E2
:103CB00014F0800F144B05FA02F205D0D3F810155A
:103CC0000A43C3F8102570BDD3F814150A43C3F88E
:103CD0001425631E062BF6D8EFF31186202383F3F9
:103CE0001288BFF36F8F2046FFF788FE204604F04E
:103CF0002AFA064A1368854023EA0503136086F30F
:103D00001188BFF36F8FDEE700700240F8180020C3
:103D1000030610B5044605D4FFF712FE10B1204685
:103D2000FFF76CFE014BC3F8184510BD0070024050
:103D3000084B70B5C31A0D4607499B1004465943FA
:103D40000648402204F02BFA2B4601462046BDE8E7
:103D50007040184718190020B76DDBB608900000B6
:103D600073B50C4C0C4A4023041B00930D460B46C4
:103D70000A49A41061430646094804F03CFA011EB2
:103D800005DA30462B4602B0BDE87040184702B055
:103D900070BD00BF1819002061820000B76DDBB64E
:103DA0000890000010B5EFF31184202383F31288EC
:103DB000BFF36F8F074A136823F00201DB0711601E
:103DC00002D4012004F03EFC84F31188BFF36F8F0E
:103DD00010BD00BF68190020002270B50121044603
:103DE0001046FEF705F90F4801F066F80E4B9842B1
:103DF00015D101F071F826690C49304603F0B9FE7F
:103E000000280BDB012535642469084904F11C00F6
:103E100003F0AFFE002801DBE564002070BD6FF009
:103E20000400FBE7293F00000000AD0BAC9200004E
:103E30001FB500220123CDE90223094ACDF800D0A5
:103E40006B46CDF804D004F004FA002805DB4FF4EB
:103E500080420023684602F001F805B05DF804FBDB
:103E60007F82000030B4104B0C2202FB003301466D
:103E70000020D3E90E529863EFF31180202484F3DD
:103E80001288BFF36F8F1C6C04F0C00444F002046E
:103E90001C6480F31188BFF36F8F1DB12B4603485C
:103EA00030BC184730BC704718190020089000003B
:103EB00010B4EFF31182202383F31288BFF36F8FC6
:103EC0001748016841F002040460C80707D482F370
:103ED0001188BFF36F8F012010BC01F015B84FF0AF
:103EE0008041D1F80C04D1F80C14C907EFD5EFF3D9
:103EF000118083F31288BFF36F8F0A490B6C03F0B4
:103F0000C00343F002030B6480F31188BFF36F8F8B
:103F100082F31188BFF36F8F002010BCFFF7A2BFA0
:103F2000681900201819002010B1012804D070472A
:103F3000034B1B6C5B0701D1FFF794BF704700BFB9
:103F400018190020024AC3B21C2003FB002070474E
:103F5000181900202DE9F0413849BFF35B8F07465F
:103F6000012251E8003F41E800200028F9D1BFF3C9
:103F70005B8F33B9324933484B60CB608A6003F0C2
:103F80000BFE7B1E012B2BD8012F07D14FF0804356
:103F9000D3F81C3403F00303012B21D004F080FD7F
:103FA0000546F8B9284B1B78E3B14FF08043022255
:103FB000C3F808230646DFF894804FF08044D4F815
:103FC0001824D4F81834D20315D503F00303012BB9
:103FD00001D0012F0FD155B386F31188BFF36F8F36
:103FE000BDE8F081EFF31186202383F31288BFF33D
:103FF0006F8F0125DFE7ADB1304604F02CF8D4F81F
:104000001835002BDBD1D4F80421002AD7D0C4F80E
:104010000431D4F804310123C4F81835C8F88031CC
:10402000A360CCE70021212002F09EFBE7E74FF0E0
:1040300080430222C3F80423D2E700BF14190020F2
:104040000419002034190020F21B002000E100E0D8
:1040500008B5074804F09EFB38B10648FEF7D2F9D0
:104060000448FCF7FFF9002008BD6FF01200FBE7E1
:1040700044900000794000000A2838B5074D0446F6
:1040800004D1AB680D215B6828469847AB680348AC
:104090005B68E1B29847204638BD00BF44900000FD
:1040A000F0B54068057B01F01F0444EA451405693A
:1040B00087B0002D64D0B2F5001F00F1100506D1C5
:1040C0002146284604F03EFB002007B0F0BD01AEBB
:1040D0000027B2F5800F0197776039D1B3F1007FE7
:1040E00014BF052304238DF804300023CDE90463B5
:1040F0000393836823FA01F111F001011AD1B2F19F
:10410000A07F17D104F01F03620903F5E0732AD0E2
:10411000012A3BD11F4A52F82330DB070AD40DF1A4
:10412000030632462146284601F0CCF91A4B984244
:104130001CD0029603AA2146284601F085F8174BA9
:10414000984220D101222146284601F01FFABBE700
:10415000B3F1C06F05D0B3F1007F14BF0123022378
:10416000C1E70323BFE74FF0A042D4E7314628461A
:1041700001F006FA094B9842DBD06FF00B00A4E780
:104180006FF08500A1E76FF015009EE751F823302E
:10419000FFDE00BF000300500400AD0B0000AD0BBC
:1041A00038B545682B69B3B11035284601F0D8F908
:1041B000044680B90146284601F09EF9084B984212
:1041C0000BD108492246284601F076F922460521FE
:1041D0000620FDF70DFF002038BD6FF00400FBE75F
:1041E0000000AD0BE9410000420970B5034602D062
:1041F000012A17D070BD0D4E326951680029F9D0DF
:1042000003F01F0301250C689D400029F2D08A6845
:104210002A4002D04B68304698472CB1236821468B
:104220001C46F2E7024EE7E72346F8E7309000002D
:104230001C9000002DE9F043466840F20635D00698
:10424000337B87B002EA050554BFC2F34010032058
:1042500001F01F07B5F5837F144647EA43178DF831
:10426000030045D00FD8062D18D007D8B5B1022DC0
:1042700040D06FF0150007B0BDE8F083B5F5807F42
:10428000F7D101250AE040F20222954234D0B5F57B
:10429000407F33D0B5F5007FEBD102250123220307
:1042A00003FA01F12CD57368C3F80815326982BB93
:1042B00007F01F037F0929D0012F77D13E4A02EB77
:1042C000830284F48033D2F80017C3F30043C4F3AD
:1042D000404444EA430421F4E16144EA800421F0CB
:1042E000070144EA05230B43C2F800370020C2E768
:1042F0000725D3E70425D1E70525CFE70325CDE73B
:10430000630344BF7368C3F80C15CFE74FF0A042B6
:10431000D5E710360DF102023946304601F0D2F8E9
:1043200014F4403F80460CD13946304604F008FA78
:10433000224B9845DAD19DF80210304601F01AF967
:10434000D4E701AB4FF0000903AA39463046CDE966
:104350000439CDE90199CDF80C9000F075FF174BA9
:10436000984286D114F4003315D09DF803308DF8AF
:104370000E3084F48034C4F300444B4603AA39461B
:1043800030468DF80C508DF80D4001F017F80B4BAE
:104390009842CDD06DE7CDE9043303AA0DF10303B4
:1043A00039463046039300F04FFFF0E703F5E07322
:1043B00052F82330FFDE00BF000300500000AD0BB9
:1043C000036803F01F025B09026004D0012B03485D
:1043D00018BF002070474FF0A04070470003005006
:1043E0002DE9F04FDFF86091DFF860A185B0154648
:1043F000834600EB810140F2FF18594503D10020AC
:1044000005B0BDE8F08FDBF800305804C3F3C322D9
:10441000C3F3080400F191801B0E19F802704445A3
:1044200008BF4FF0FF34192B00F28A80DFE803F059
:104430000D141A1D20261D88888888366388888870
:10444000888888888888667C7F82C5F80C45621CCD
:104450005ED10BF1040BD0E7C5F81445631CF8D00E
:1044600000265FE0C5F80845F1E7C5F81045F5E717
:10447000661CC5F80845ECD0002604E0601CC5F8B1
:104480000C45E6D0012603A80394FFF799FF039B90
:10449000012202FA03F3C0F80C3508E0C5F808451C
:1044A000002FDBD1631CD4D0002632460627DBF870
:1044B0000030019303F40040002818BF002203A835
:1044C000009218BF01260394FFF77AFF039C019B1B
:1044D000009A00EB8400C3F3412CD0F800473B0264
:1044E00043EA8C03134304EA0A04234343EA4603E2
:1044F000C0F80037ADE7C5F80C45D1E7C5F8604511
:10450000621CDBF80030A4D0C3F30043002BB9D009
:1045100003A80394FFF754FF039B012606FA03F355
:10452000C0F808353246C2E7C5F86445E8E7C5F883
:104530006845E5E7C5F86C45E2E76FF015005FE711
:104540006FF085005CE700BFA8950000F0F8FCFF65
:104550002DE9F041044647680D4604F0A1FA4FF0FA
:10456000200888B9264B1B7873B16426606803F075
:10457000A9FFF0B9012004F057F8013EF6D100215F
:10458000212002F0F1F8F0E7EFF31186314688F3CD
:104590001288BFF36F8F606803F094FFA8B986F3A9
:1045A0001188BFF36F8FEFE786F31188BFF36F8F2A
:1045B000E5E7EFF31186314688F31288BFF36F8F7A
:1045C000606803F07FFF0028EED0BB691D70636850
:1045D000BA691B680020C3F844250122C3F84825A6
:1045E000C3F82001D3F82041C3F85801D3F858018B
:1045F0009A6081F31188BFF36F8FBDE8F08100BF2F
:10460000F21B0020F7B50546002201210220FDF72C
:10461000EFFC0220FDF7BCFC6A6811681369C1F861
:104620002435137D507D927D03431343C1F86C35CF
:104630006E68D6E9004313F0010348D02F6907F1F3
:104640000C0003F0FDFF304B98425AD1387B04F147
:104650000C0204F5907103F0E9FF387B012707FA9B
:1046600000F000F0C1FB0823C4F80035B369C4F8BA
:1046700044350023C4F84835A760D4F85831002BDE
:10468000FBD00021C4F800156B68DC6801AA204645
:1046900003F061FE002805DB019B22681979186888
:1046A000FFF79EFE6A6813680821C3F80015117AA7
:1046B00051B9D269C3F834250122C3F83825C3F8AB
:1046C0001011D3F810111A60002003B0F0BD0822B9
:1046D000C4F80025B269C4F84425C4F8483501235C
:1046E000A360D4F82031002BFBD00023C4F8203184
:1046F000D4F820310123E3604FF48073C4F804330D
:10470000BBE76FF00400E0E70000AD0B70B50123DC
:1047100083400E4ABFF35B8FDC4352E8001F01EA7F
:10472000040542E80056002EF7D1BFF35B8F4FF42B
:10473000803282400648C0F80823BFF35F8FBFF382
:104740006F8F0B4214BF0120002070BD881900201C
:104750000010014070B40E49D1E90034D01AC318DA
:1047600044F1000422F07F46C1E90034A6F50013AD
:10477000B3F5400F09D2074B1B681A0A1B069C1998
:10478000054B42F10005C3E9004570BC02F0A0B939
:10479000180500208C1900202005002011B3BFF35C
:1047A0005B8F0123104A834052E800CF4CEA030C90
:1047B00042E800C10029F7D1BFF35B8F0B4A4FF4E9
:1047C00080338340C2F80433094BBFF35B8F1B680F
:1047D000BFF35B8FC340DB0742BF064B4FF4003291
:1047E000C3F80021704700BF881900200010014065
:1047F0008419002000E100E00D4B1868010A000652
:10480000BFF35F8F0B4BD3F80435181841F100014B
:10481000B3F5801F0AD2084BD3E90023904271EB15
:10482000030303D210F1807041F10001704700BF13
:104830008C19002000100140200500202DE9F04FC8
:1048400085B016461F469DF840A00446FFF75EFF60
:104850000190FFF7D1FFB04271EB070354D23E4BFA
:10486000301A67EB0101984271F100014FD23B4BC6
:1048700003EB0413D3E902239F4208BF96425ED0A4
:1048800037494FF4803804F1500508FA04F8AD00B8
:10489000C1F848832046ADB203F0AEFE26F07F4B50
:1048A00005F1804504F5A87305F58835DC464FF021
:1048B00003090293029A2CF07F4341F82230C1F899
:1048C0004483D1F80435274A6FF00200C01A6044CF
:1048D00020F07F40904232D9286868B1D1F8043581
:1048E0000393A3EB0B0020F07F40B0F5000F26D917
:1048F000204603F081FE039BBAF1000F07D109EBBC
:10490000030C09F10109D5E7BAF1000F09D06FF0E6
:10491000150520460199FFF741FF284605B0BDE87F
:10492000F08F0123104ABFF35B8FA34052E8000FC2
:10493000184342E800010029F8D1BFF35B8F074913
:104940000E98230101EB0412C8500F9B5360C2E97B
:1049500002670025DDE700BF010080000805002098
:1049600000100140FDFF7F00841900207FB51C4C22
:104970001C4BC4F80833C4F848331B4B00254FF0D8
:10498000FF304FF0FF31C4F80855C3E902014FF47E
:104990008033C4F80433154B02264FF40032012152
:1049A000C4F804631120C3F880212A46FDF720FBD8
:1049B0001120FDF7EDFA0E4A0123A3602360136076
:1049C0000C4B0D4A0093CDE9015500232846FFF713
:1049D00035FF3046FFF7BEFA284604B070BD00BF71
:1049E0000010014003000F000805002000E100E076
:1049F0008819002055470000FFFF7F002DE9F7438D
:104A00002F4CD4F8043399070BD5D4F8043143B1B3
:104A10002C4A0023C4F80431D4F80431136801335C
:104A20001360D4F80433DA0329D5BFF35B8F264B28
:104A300053E8002F22F0010143E800100028F7D1CD
:104A4000BFF35B8FD30702D4D4F84031BBB100254C
:104A5000C4F84051D4F84031FFF7CEFEEFF3118295
:104A6000202383F31288BFF36F8F184BD3E90267BB
:104A7000B042B94106D282F31188BFF36F8F03B001
:104A8000BDE8F0834FF0FF384FF0FF39C3E90289EA
:104A9000D3E900101D604FF48033C4F84833C4F8E4
:104AA0004051D4F8403182F31188BFF36F8F002951
:104AB000E5D0009032463B4628468847DFE700BFF6
:104AC000001001408C1900208419002008050020E6
:104AD00030B5431C124C85B005D08442A8BF0446B3
:104AE000012CB8BF0124FFF787FE0E4B0C4DD3E914
:104AF0000013401AB0F5000F10D22218AA4228BFA6
:104B00002A4652184FF0000007490091CDE90100F4
:104B100043F10003FFF792FE05B030BD2A46F0E7EF
:104B2000FFFF7F00180500205547000008B5FFF77C
:104B300063FE024B1B68C01A08BD00BF18050020A9
:104B4000BFF34F8F0549064BCA6802F4E062134376
:104B5000CB60BFF34F8F00BFFDE700BF00ED00E06B
:104B60000400FA054FF08053D3F83021082A06D10B
:104B7000D3F83431052B02D8024AD05C70470020AC
:104B8000704700BFC4950000024AD2F80034002BE1
:104B9000FBD0704700E0014010B54FF08053D3F8D0
:104BA0003021082A4ED14FF080420021C2F80C116A
:104BB000C2F81011C2F8381502F54042D3F80414B7
:104BC000C2F82015D3F80814C2F82415D3F80C1431
:104BD000C2F82815D3F81014C2F82C15D3F8141401
:104BE000C2F83015D3F81814C2F83415D3F81C14D1
:104BF000C2F84015D3F82014C2F84415D3F8241491
:104C0000C2F84815D3F82814C2F84C15D3F82C1460
:104C1000C2F85015D3F83014C2F85415D3F8341430
:104C2000C2F86015D3F83814C2F86415D3F83C14F0
:104C3000C2F86815D3F84014C2F86C15D3F84434A0
:104C4000C2F87035FFF78EFF18B13F4B3F4AC3F8EB
:104C50008C26FFF787FF18B13D4BFB22C3F81825C0
:104C6000FFF780FF70B14FF080414FF08053D1F8D3
:104C7000E42ED3F8583222F00F0203F00F0313434F
:104C8000C1F8E43EFFF76EFF20B1324B4FF40072E3
:104C9000C3F840264FF08053D3F83031082B1AD197
:104CA0004FF08043D3F80024D20744BF6FF00102D5
:104CB000C3F800244FF08053D3F83431052B02D8C9
:104CC000254AD35C3BB14FF01023D3F808224FF0B4
:104CD0008043C3F858254FF01021D1F80C32DB0780
:104CE00014D51E480123C0F80435FFF74DFFD1F855
:104CF0000C3223F00103C1F80C32FFF745FF00230B
:104D0000C0F80435FFF740FFFFF71AFFD1F8003273
:104D1000002B03DBD1F80432002B14DA0F490123F6
:104D20004FF01020C1F804351224FFF72DFFC0F812
:104D30000042FFF729FFC0F80442FFF725FF0023D8
:104D4000C1F80435DEE710BD005000404881030083
:104D500000F0004000900240BE95000000E00140DD
:104D600030B50468CCB1BFF35B8FB4FA84F3C3F100
:104D70001F03DBB201229A4024EA020250E8005FDE
:104D8000A54204D140E8002CBCF1000FF6D1BFF3DE
:104D90005B8FE6D102480B7030BD0248FCE700BFD4
:104DA0000000AD0B0200AD0B10B50368CB40DB0774
:104DB00014D401238B400268BFF35B8F43EA0201E6
:104DC00050E8004F944204D140E8001CBCF1000FB1
:104DD000F6D1BFF35B8FEED1014810BD0148FCE76F
:104DE0000000AD0B0400AD0B014BC3F80405704788
:104DF00000F00140F7B5044618B1012823D003B0F4
:104E0000F0BD4FF080430222C3F808230122DA608C
:104E1000C3F80401D3F80431064601238DF80730A6
:104E200042F210754FF08047D4B1012CE7D1D7F88A
:104E30000C3403F48033AEBB83B3012003F0F4FBE6
:104E4000013DF4D12AE04FF080430022C3F808036B
:104E50005860C3F80021D3F800310DF10706DCE7F4
:104E6000D7F8183403F480333EB9002BC7D00120A3
:104E700003F0DAFB013DF3D1C1E7D7F8182402F0C3
:104E800003023260002BBAD09DF80700012803D13D
:104E900003F0CAFB013DC7D1012CB0D1054B002264
:104EA0005A71ACE7D7F80C2402F001023270002BE3
:104EB000EAD1F3E790190020044B1A7922B90122B4
:104EC00018609A8002487047024870479019002085
:104ED0000000AD0B0C00AD0B08B5094B1B682BB1E6
:104EE0000020FDF777F808B9FDF752F84FF080433E
:104EF0000022C3F81825034B01221A7008BD00BF19
:104F000090190020F01B002010B510B1012843D0EB
:104F100010BD4FF08043D3F81814D3F81824C803F9
:104F200021D502F00303012B04D013B10020FFF7B9
:104F300061FF00234FF080420220C2F8183508229A
:104F40004FF4827303F180430021196002F1804223
:104F50001C6801241460154A12680AB34FF080439C
:104F6000C3F80403D4E7D3F81424D107E1D5D3F868
:104F70001C249207DAD40D4A12681AB10222C3F82F
:104F80000423C5E7D3F80421002AFBD00022C3F88C
:104F90000421D3F80431BBE700224FF48073D1E73A
:104FA0001A68002AFCD019601B68B1E7901900202C
:104FB00010B54FF08043D3F800216AB10022C3F846
:104FC0000021D3F800210122C3F80823114B58799E
:104FD00010B95A711B6898474FF08043D3F80421E9
:104FE00072B10022C3F80421D3F80421D3F81824A5
:104FF000D3F81824920704D10122C3F818259A6027
:1050000010BD0222C3F80823024BBDE810401B6804
:105010000120184790190020036803F01F025B0964
:10502000026004D0012B034818BF002070474FF0E6
:10503000A040704700030050034A430900F01F00DE
:10504000D35C1844C0B27047CA95000070B50546DD
:10505000FFF7F2FF0C4C08300E4634F81030DA053A
:1050600008D5C3F3432304EBC302284654F8333076
:1050700052689847A3682BB1E26831462846BDE8DC
:105080007040184770BD00BF6001002008B5FFF7F1
:10509000D3FF034B083033F81000400B08BD00BFAE
:1050A0006001002008B5FFF7C7FF034B083033F855
:1050B0001000C0F3400008BD6001002008B5FFF7F4
:1050C000BBFF034B083033F81000C0F3401008BD9D
:1050D00060010020034611F0010010B5CCB20DD1E3
:1050E000A207C4F3400012D5094AD2F8200558603F
:1050F000C2F82005003818BF012008E04FF0A04199
:10510000D1F820251A60C1F82025002AE8D010BD6A
:105110000003005010B5FFF78FFF124A083032F835
:105120001030D9051CD5C3F3432123F4F85322F8DA
:10513000103002F10E04002034F8023F13F4807F97
:1051400003D0C3F3432399420AD001303028F3D16E
:10515000002342F831300448BDE81040FFF724BE78
:1051600010BD00BF60010020D8010020F0B5054649
:1051700000200446012607468C420BD1114BD3F880
:105180007C2132B10022C3F87C21D3F87C3140F07D
:105190000040F0BDE3B29B0003F580729B0806FA65
:1051A00003F31D420BD002F1804202F5C042D2F857
:1051B00000C0BCF1000F02D0176012681843013420
:1051C000DAE700BF00600040F7B506460846FFF783
:1051D00033FF194F00F108050C4637F81530DB078F
:1051E00027D5304603F088FA2046FFF767FF40B125
:1051F0002046FFF74BFF316800F5A270002341F80D
:1052000020302046FFF786FF002301A827F815303D
:105210000194FFF701FF019B00EB8300074BD0F8DF
:105220000027134043F00203C0F80037044803B0DE
:10523000F0BD0448FBE700BF60010020F0F8FCFF70
:105240000000AD0B0400AD0B2DE9FF411646804672
:105250000846FFF7F1FE0D463168044609B32846BB
:10526000FFF720FF18B12846FFF728FF10BB0023E7
:10527000CDE900338DF80E308DF80F300DF10F02AF
:105280000B4628460DF10E0103F0DEF9474A04F102
:10529000080132F8113023F0020343F0010322F831
:1052A0001130736863B328461F785968FFF7FAFE18
:1052B00010B1D1B13E4826E03C4A04F1080032F872
:1052C000103023F02003DB04DB0C22F8103061B136
:1052D000032FEFD87168496891F800C0D8F8001022
:1052E000A7B90CF5A27C41F82C70304A04F10801F2
:1052F00032F8113023F01C0343EA870322F81130FF
:10530000B3684BBB2B4804B0BDE8F08101EB8C01C6
:1053100043EA4C33D1F810E52EF0030EC1F810E546
:10532000D8F8001001EB8C0E43F02003DEF81015C6
:1053300022F8103021F44F3121F44071CEF81015CD
:105340002902DEF8108501F47C5141EA074141EA67
:105350000801CEF81015C8E7D3E900672846FFF723
:10536000D9FE002ECED0114DD5E90023964203D1AF
:105370009F4201D1002209E00F480DF10F01FFF714
:10538000EFFC0C4B9842BED19DF80F2045F83260DF
:1053900005EBC20308345F6035F8143043EA42235A
:1053A00043F4807325F81430ACE700BF600100209F
:1053B0000400AD0B0000AD0BD80100202DE9F04337
:1053C0000C4685B08046204611461E46FFF734FE47
:1053D000054629B32046FFF765FE18B92046FFF7BA
:1053E0006DFE18BB314F05F1080937F8193013F07D
:1053F0001C0F02D04B78012B18D001238DF80F30F1
:105400000023CDE900134A1C8B1C20460DF10F012F
:1054100003F01AF937F8193043F0030327F819306D
:10542000002E41D02046FFF73DFE18B9204805B0B8
:10543000BDE8F08396F800C0D8F800301B4F0CF59B
:10544000A272002143F8221005F1080237F8121069
:1054500021F02001C904C90C27F8121075781DB37A
:10546000D8F80000B67800EB8C002D04D0F8103589
:1054700023F4991323F4F853C0F81035230203F4EE
:105480007C5305F440353605D0F810E52B4306F47F
:10549000801641EA4C31334341F0200143EA0E03C8
:1054A00027F81210C0F810350248C0E7600100204C
:1054B0000400AD0B0000AD0B014BC3E902127047B5
:1054C0006001002010B508461446FFF7F7FD50B103
:1054D0000846FFF7B1FD054B083033F8103004489B
:1054E0005B0B237010BD0348FCE700BF6001002088
:1054F0000000AD0B0400AD0B70B5164D95F8804063
:1055000006462CBB2146602205F1100003F0BFFCCB
:1055100030682E6F21468E420ED10023C0F87C31B8
:10552000D0F87C3140F30730FCF732FD01230A4804
:1055300085F88030AB6770BDCBB29B0003F58072FD
:105540007C2B08BF845001F1010108BF8358E2E7BA
:105550000248F0E7600100200000AD0B0C00AD0B2D
:10556000034B93F88000003818BF0120704700BF3C
:10557000600100200148FFF717BC00BFD4010020E4
:105580000148FFF7EDBB00BFD401002073B50368ED
:105590001646D3F80423002AA8BF4FF00042054660
:1055A000A8BFC3F8042308460C46FFF787FD00B3E5
:1055B0000846FFF777FD0146D8B92046FFF766FD9C
:1055C00004B2A40004F5807203462868815029685B
:1055D00082582144D1F8102542F00102C1F810256B
:1055E0002EB12968012202FA03F3C1F8043302B094
:1055F00070BD2046FFF720FD0F4B083033F8103008
:10560000C3F38203042B12D0052B12D001A80194FE
:10561000FFF702FD019AD0F81035D34003F00103E3
:10562000991C204602B0BDE8704003F056B8032133
:10563000F7E70221F5E700BF600100202DE9F04FF8
:10564000694BDFF8A881D3F80403D8F87010C0B212
:1056500089B040F00040FFF789FD051E2FDAC246F1
:1056600000235AF87C1F06A8CDE90633FFF732FD68
:105670005F4B01930DF118094FF0000B019A12F8DE
:10568000013B0192DA0803F007031AF8022022FA1C
:1056900003F3DA071CD409F10409BBF1000F14D09D
:1056A000D8F870104FF00040FFF760FDD8F87C107C
:1056B00006A8FFF70FFD0028DAD125F000450124E8
:1056C000002D79D109B0BDE8F08F4FF0010BD5E77F
:1056D000484B5B440293D9F800100029DBD0029BB1
:1056E00091FAA1F11C78B1FA81F141EA4414204603
:1056F000FFF7A2FC0830059438F81070C808BB0802
:1057000019F80020039301F00701012303FA01F1C6
:1057100022EA010209F8002005A8FFF77DFC059A9E
:10572000039B02F5E072C7F3820650F822205B0764
:105730003746C2F3014224D520463946D6B2FFF798
:1057400085FC05A80594FFF767FC059B03F5E0734E
:1057500050F82330C3F301439E4207D10021204675
:1057600002F0BBFF3146204602F0B7FF05A80594C2
:10577000FFF752FC059B012202FA03F3C0F8203523
:10578000A9E7022A0CD10321204602F0A6FF06F069
:105790000503012BEAD139462046FFF757FCE5E720
:1057A00002212046039202F098FF032EF3D0039AC1
:1057B000032ADBD1022EEDE795FAA5F3B3FA83F3C2
:1057C00004FA03F29B0003F1804303F5C04325EA8A
:1057D0000205D3F81005D3F81015C0F30520C1F366
:1057E0000141FFF733FC6BE70060004060010020DF
:1057F000DA950000DA95000010B5184C237853BBF9
:105800000278C2F34003920712D54FF08053D3F8C9
:105810003021082A0BD1D3F83431052B07D8104A90
:10582000D35C23B14FF080430122C3F83826012313
:105830004FF08042C2F88035037803F00103C2F8CC
:1058400078350020FCF7C6FB08B9FCF7A1FB012363
:105850000448237010BD0448FCE700BFF11B002082
:10586000DC9500000000AD0B0C00AD0B4FF0804349
:105870004FF46072C3F80823014B00221A6070478E
:105880009819002008B5FFF7F1FF03680BB1014A32
:10589000136008BD9819002010B54FF08043D3F86D
:1058A0000443620707D54FF4847002F04DFF10B136
:1058B0001E4B1B689847A30608D54FF48A7002F068
:1058C00043FF18B11A4B00201B689847600608D5A3
:1058D0004FF48C7002F038FF18B1154B01201B6893
:1058E0009847210608D54FF48E7002F02DFF18B1AD
:1058F000104B00201B689847E20508D54FF49070C4
:1059000002F022FF18B10B4B01201B689847A3053A
:105910000AD54FF4927002F017FF28B1054BBDE88D
:1059200010401B680220184710BD00BFA0190020BE
:105930009C1900209819002001460148FFF710BA71
:10594000E401002038B5EFF31185202383F312889A
:10595000BFF36F8F064B9C6802F02FFF85F3118811
:10596000BFF36F8F2046BDE83840FCF795BA00BF03
:10597000A419002038B5094B53F82040013053F8E2
:105980002050A54200D838BD636823B1204602F0FC
:1059900017FF0834F5E723689847FAE7C09300003B
:1059A00070B52B4B2B4C2C4D012286B003201A7066
:1059B000FFF7E0FFFBF776FF02F01EFF0420FFF782
:1059C000D9FF2646AE4204F1300410D300F00EFE9B
:1059D000204C224EAC4226D300F01CFEFAF702FD0A
:1059E0001F4A137B23F00103137306B070BD54F8F4
:1059F0000C3C059354F8103C049354F8143C039366
:105A000054F8183C029354F81C3C019354F8203C81
:105A1000009354E90A2354E90C0100F0A9FB54F85F
:105A2000303C5E65CDE7D4E90A23B3F1FF3F08BF00
:105A3000B2F1FF3F05D052EA0301206803D103F021
:105A400038F83034C6E73146183000F0C7FFF8E7C1
:105A5000F21B0020EC910000EC910000E18B0000B3
:105A6000A805002008B50348034A0021121A02F0D5
:105A7000BFFE08BDC8030020F41B002070B5002342
:105A800086B00122CDE90423134E144D01930F2259
:105A9000CDE902321249142303FB005506EBC01670
:105AA00004464FF4C07000FB04110E4B00954FF4F8
:105AB000A072304600F05CFB737B0B4AEE6023F073
:105AC000040373734FF4046304FB033313442C7413
:105AD0006B6006B070BD00BF28050020A41900202F
:105AE000C02C00209588000080240020BFB5002035
:105AF000FFF740FF2C4B83F308882C4D2C4E6B692D
:105B00002C4F43F400736B610024E02385F82230AE
:105B1000EC772C766C76AC7685F820406B6A43F493
:105B2000E0236B6285F82340FCF732F9FCF7E8FAD2
:105B30004FF0FF33AB62EB62FCF7A8FBFCF704FB12
:105B40001D4BB36040F201129A81C3E91844DC6630
:105B500002F01FFE0120FFF70DFF0220174DFFF797
:105B600009FF00F077FD164B756105930123154978
:105B70000094CDE903434FF480623B46CDE90144F4
:105B8000284600F0F5FA6A7B064622F00402284611
:105B90006A7302F0CAFF2046FFF770FF3A463146AB
:105BA0002846FCF78BFA00BFC02C002000ED00E077
:105BB000A4190020A159000028060020A8050020F3
:105BC000E2950000402E002038B5064C064D00201E
:105BD000AC4200D338BD204602F00FFE0028F9DBAE
:105BE0001C34F5E75C0200207802002073B50C46F7
:105BF000EFF31181202585F31288BFF36F8FC568FD
:105C00005DB125602B68C360836901338361002027
:105C100081F31188BFF36F8F11E052EA030603D1BD
:105C200025606FF00B00F3E7CDE900230246083052
:105C300000F028FC18B9034B9B685B69236002B035
:105C400070BD00BFA41900202DE9F341044617469A
:105C50001E46EFF31188202383F31288BFF36F8F62
:105C6000C368334A7BB180689168884219D057EA8B
:105C7000060318D188F31188BFF36F8F6FF00F0000
:105C800002B0BDE8F081916891F90E1021610133F5
:105C9000E3609368A36088F31188BFF36F8F0020DF
:105CA000EEE72169F2E791F90E1090F90E30994272
:105CB000A8BF19466FF07E029142B8BF11468B42D1
:105CC0002DDD02F0F2FD0546CDE9007619482246A9
:105CD000414600F0D7FB0028E1D0EFF311862023E6
:105CE00083F31288BFF36F8FA068D0B12368216956
:105CF0009C420AD04BB193F90E309942A8BF194685
:105D00006FF07E039942B8BF194602F0CEFD40B154
:105D10000848314600F026FC6FF00A00B0E7002585
:105D2000D2E7002DF4D186F31188BFF36F8FF3E72C
:105D3000A4190020F31B002038B58368044663B320
:105D4000194A926893422BD1C368012B03D9013BB6
:105D5000C360002038BDEFF31185202383F3128840
:105D6000BFF36F8F0169806802F09FFD204602F04B
:105D70003BFFA06058B190F90E202261002282679B
:105D800002F0D3FE0948294600F0ECFBE1E7E060B1
:105D900085F31188BFF36F8FDBE76FF01500D9E74C
:105DA0004FF0FF30D6E700BFA4190020F31B0020FE
:105DB00037B51146EFF31185202282F31288BFF325
:105DC0006F8F04689CB12368426823F003039442F8
:105DD000036008BF43600121204602F0D6FD04465F
:105DE00085F31188BFF36F8F204603B030BD51EAB1
:105DF0000302F5D000F10802CDE900131046294650
:105E000000F040FB0028EFD1014B9B685C69EBE799
:105E1000A419002038B50446EFF31185202383F33D
:105E20001288BFF36F8F02F0DFFE48B10022826755
:105E300002F07BFE29460848BDE8384000F092BBDE
:105E4000D4E902329A4218BF0133A36085F3118866
:105E5000BFF36F8F38BD00BFF31B002013B5EFF306
:105E60001181202484F31288BFF36F8F846844B1BA
:105E7000013C846081F31188BFF36F8F002002B072
:105E800010BD52EA030406D181F31188BFF36F8F6E
:105E90006FF00F00F3E7CDE900230246014800F060
:105EA000F1FAECE7F31B00202DE9F043DFF8348131
:105EB00085B005464FF0FF364FF0FF37EFF31189FD
:105EC000202383F31288BFF36F8FD5F880408CB9FD
:105ED000022105F1980002F07BFD002860D100232B
:105EE000CDE90067029305F1880249463E4800F07B
:105EF0007DFCE3E7D5F884202368C5F88030944220
:105F000008BFC5F88430D5F8983043F00203C5F8CF
:105F10009830E36823F0040343F00103E36063680F
:105F200089F31188BFF36F8F20469847EFF31189EB
:105F3000202383F31288BFF36F8FE368D90623F021
:105F4000010237D4E260E3689A071AD5D8F8000056
:105F500023F00203E360A0B10268002188B1436826
:105F60009C4237D1036869BBD8F80420C8F80030D8
:105F7000824201D1C8F80430002340F8083BFFF703
:105F800049FFD5F8983023F00203C5F8983089F31B
:105F90001188BFF36F8FDB0590D400F063FB8DE7B2
:105FA00005F1900400220121204602F076FE00282F
:105FB000F8D194E723F01103E36004F11000FFF738
:105FC00029FFC0E70B60D8F80430834208BFC8F847
:105FD0000410D1E722B11368014610461A46BDE706
:105FE0001346F9E7C4190020F31B0020F8B5C36875
:105FF0009A0704460F46C3F340062CD45B071AD415
:106000000B680BB983680B60E368DD0744BFA368C6
:106010003B603D684CBF02260126002D3AD01F4B45
:106020009B68AB420AD0D5F89830D807C3F38002FA
:1060300014D46FF0120600233B6025E002F030FD1F
:10604000D5F898300028F0D1D907C3F3C002F0D5B5
:1060500052B15B0708D46FF00F06ECE7002AFAD1C3
:10606000C3F3C003002BF6D100232360D5F884309E
:1060700063B9C5E92044284602F0B5FCE36843F063
:106080000403E3603B68A3603046F8BD1C60C5F8BC
:106090008440F0E76FF01506CDE700BFA41900209B
:1060A000F0B589B004460020C4E920000E9D04F13B
:1060B0008800C4E9220004F19000C4E924004DB333
:1060C0002879002840F2011008BF0120C4F8980088
:1060D00000204FF0FF364FF0FF37CDE90330CDE918
:1060E0000100CDE906670C4B0094204600F08CF8C7
:1060F00055B1296811B1204602F0D8FC6B791BB16B
:10610000237B43F001032373204609B0BDE8F04030
:1061100002F0CFBC0120D9E7A95E000037B501909D
:106120000846EFF31184202181F31288BFF36F8FAB
:10613000C16811F01E0F16D153EA020508D101A95A
:10614000FFF754FF84F31188BFF36F8F03B030BDA6
:1061500041F00801C160019981621030034900F0EB
:106160003DFC0120EEE70020ECE700BFF5890000D0
:106170002DE9F043073285B022F007020E461F4694
:106180001099017300F158037F32C0E916330446B9
:10619000002322F03F020421836041733F2A0F98BD
:1061A000A073C4E90633E37306F14009A2F1400885
:1061B00005D883F31188BFF36F8F084602DFB51847
:1061C00029462046FBF76CFC07300E9B20F00700A9
:1061D000A066C4E9189802930D9B01932D1A0C9B9D
:1061E00000932A463B4631462046FBF735FF002305
:1061F0006365044B9B6803B1DB6EE366284605B01C
:10620000BDE8F083A4190020F0B587B000250595FE
:10621000109D04950F9D03950E9D0295DDE9127664
:106220000D9D01950C9D00950446FFF7A1FFB6F169
:10623000FF3F08BFB7F1FF3F05D056EA070305D17E
:10624000204600F0A1F9204607B0F0BD03493A46C8
:10625000334604F1180000F0C1FBF4E7E18B0000C5
:1062600038B50D4D2B4653F8184F9C4200D004B959
:10627000EC68AB6838B95A7BD20604D1A26912B96E
:10628000DA897F2A05D89C4202D0204600F0EEFA37
:1062900023466B6138BD00BFA419002008B590F9F2
:1062A0000D20437B002A014604DA03F07F03437389
:1062B00002F001FC044B9868431A58425841BDE86B
:1062C0000840FFF7CDBF00BFA419002070B490F9BB
:1062D0000D30427B002B29DBD30627D183692BBBF2
:1062E000134962F07F0242730A4652F8184F9442F3
:1062F00018BF2346CC6923B9C0E900242060C861D7
:106300000CE090F90E5093F90E60B5420AD0AE42FF
:1063100008DD5A68C0E900321060586070BC002087
:10632000FFF79EBF9C42E7D01B68E4E770BC704754
:10633000A41900202DE9F041002A427B0E460CBF33
:1063400010210821114204460FD141EA0203D2096B
:1063500018D1437308291BD00120FFF781FFBFF339
:106360005F8F637B23F060036373274B9B68A342BB
:1063700043D1EFF30583002B3FD13046BDE8F04118
:10638000FBF7A0BD03F07F03437302F094FBE1E74A
:10639000A36813B1204602F096FB04F1180002F046
:1063A0009EFCA56D04F15807AF4211D04FF00008D4
:1063B00075B1284602F087FB05F1180002F08FFC4A
:1063C000C5F878802846FFF781FFA56DAF42EFD171
:1063D0000D4DAB689C42BFD1EFF30583002BBBD0C2
:1063E0000120FFF73DFF094BAB6040F201129A819B
:1063F0000022C3E91822DA66B1E786F31188BFF3F9
:106400006F8FBDE8F08100BFA4190020280600208E
:1064100070B590F90D20437B002A014604DA03F0A1
:106420007F03437302F047FB4B7B154A63F07F0306
:1064300010464B7350F8183FD469834208BF0023BD
:1064400023B9C1E900042160D1610CE091F90E503B
:1064500093F90E60B5420ED0AE420CDD5868C1E92A
:106460000030016059609068431A5842BDE870409E
:106470005841FFF7F5BE9C42E3D01B68E0E700BF40
:10648000A4190020F8B5124B0C461146114A986821
:106490001060DDE90676EFF31182202282F3128884
:1064A000BFF36F8F9D68284602F017FBB6F1FF3FE0
:1064B00008BFB7F1FF3F06D007493A46334605F11A
:1064C000180000F08BFA2046BDE8F840FBF7FABC54
:1064D000A4190020CC190020E18B0000F8B5044677
:1064E000EFF31186202383F31288BFF36F8F437B72
:1064F000DA0649B219D18569BDB903F07F03437348
:1065000002F0D9FA437B164A817363F07F03437329
:10651000134653F8180F984218BF0546D0695DB965
:10652000C4E900300460D46111E0A173002086F357
:106530001188BFF36F8FF8BD95F90E70B9420BD07B
:106540008F4209DD6B68C4E900531C606C60012058
:10655000FFF786FE0120EAE7A842E1D02D68DEE7DA
:10656000A419002049B9EFF3058030B9054B5A69E9
:106570009B689A4201D0FBF7A5BC81F31188BFF359
:106580006F8F7047A419002010B5EFF311842022FB
:1065900082F31288BFF36F8F427B510704D484F3D8
:1065A0001188BFF36F8F10BD22F004024273FFF712
:1065B0008DFE21460248BDE81040FFF7D3BF00BF63
:1065C000F31B0020034648B9EFF3058232B9064AAF
:1065D00051699268914201D0FBF774BC83F3118832
:1065E000BFF36F8F704700BFA4190020EFF3118134
:1065F000202383F31288BFF36F8F054B9A68D37BF8
:10660000013BD37381F31188BFF36F8F704700BFD5
:10661000A419002038B5EFF31185202484F31288E3
:10662000BFF36F8F0A4B9A68D37B0133D37300207B
:10663000FFF716FE85F31188BFF36F8FEFF311801C
:1066400084F31288BFF36F8FBDE83840FFF7BABFFD
:10665000A4190020024B03F11802C3E90622704777
:10666000A4190020F8B5EFF31185202383F31288D5
:10667000BFF36F8F19498868437B03F07F0343732F
:1066800002F019FA8B685A7B084662F07F025A734F
:1066900050F8182FCC69824208BF002222B9C3E902
:1066A00000042360CB610CE093F90E6092F90E7048
:1066B000BE420ED0B7420CDD5168C3E900210B6029
:1066C00053600120FFF7CCFD2846BDE8F840FBF7FA
:1066D000F9BBA242E3D01268E0E700BFA419002092
:1066E00050EA01032DE9F04105460E4603D1FFF7BC
:1066F000B9FF00202BE0831C71F1FF3329DB02F08E
:1067000003FB2C18EFF31188202383F31288BFF3C7
:106710006F8F124F124BB8681860FFF7BFFDB86853
:1067200010492A463346183000F058F9BA68537BAE
:1067300043F0100353734046FBF7C4FB02F0E4FA46
:10674000201A63EB0303012873F10003D1DBBDE8DA
:10675000F0816FF00104241AD4E700BFA4190020CF
:10676000CC190020E18B0000B1F1FF3F08BFB0F170
:10677000FF3F08B506D10A4B986802F0E5F94FF0E3
:10678000FF3008BDFFF7ACFF4FF47A7147F6FF7397
:106790000022C0FB0132D80B40EA4240F1E700BFC3
:1067A000A41900200C490D4A38B500244FF40045C7
:1067B0008C462146C0FB05C100236046F9F7A0FCCA
:1067C000C117FFF78DFF054A47F6FF73C0FB023480
:1067D000DB0B43EA444038BD3F420F0040420F000C
:1067E000014B9868704700BFA4190020D3B5DDE9BC
:1067F0000667089CCDE90067FFF744FE1CB1034B18
:106800009B685B69236002B0D0BD00BFA419002063
:10681000044BC01A044BC0105843044B01221A54B5
:10682000704700BFA8060020ABAAAAAAF31B00204D
:10683000C3897F2B12D80A4B1B6863B1094B90F9AF
:106840000E201B689A4209DB437BDB0606D1064B10
:10685000C31A18BF012303F0010070470023FAE7B1
:10686000D4190020D01900202805002070B50E4B47
:106870000E4C1E7C06EB460304EBC3040546204683
:1068800002F02DFA0A4B002228469A55FFF7D0FF56
:1068900048B1084B08491A68013A2046D317BDE8A9
:1068A000704000F09BB870BDA4190020A80600201D
:1068B000F31B0020D41900201168000038B5EFF355
:1068C0001185202383F31288BFF36F8F104B114A79
:1068D0009C681068A04206D1FFF7C8FF85F31188B5
:1068E000BFF36F8F38BD00211B7C11600A4AD35C57
:1068F000002BF3D02046FFF79BFF0028EED0637BF0
:10690000DB0602D12046FFF783FD2046E4E700BF07
:10691000A4190020CC190020F31B002008B506485C
:10692000064A0749121A01F065FFBDE80840054A0A
:106930000549064801F05EBF00000020C4030020A6
:1069400000960000000000000096000000000020FB
:10695000034B1B680BB9FEF7E9B80020704700BF76
:10696000D819002030B570B10B4B5B6898420AD043
:10697000036843B1D3E90421D0E90445121941EB7E
:106980000501C3E90421D0E9003213605A600023F5
:10699000C0E9003330BD00BFE801002010B50E4B48
:1069A0001C689C4204D1FFF7D3FF6FF0004010BD7C
:1069B000FFF7CEFF002CF8D0D4E904321B1A62EBAB
:1069C000E072B3F1004F72F10001EEDA002AACBFC1
:1069D00018460020EBE700BFE8010020B3F1FF3FBD
:1069E00008BFB2F1FF3FF8B504461D4616465ED01B
:1069F0008160EFF31187202383F31288BFF36F8F39
:106A0000013275F1FF3324DA2E49D1E900206FF00D
:106A100001039B1A4FF0FF3262EB00009E1B60EBFC
:106A20000500012E70F1000301DA01260020C4E9FF
:106A30000460254ED6F800C07568B44508BF4FF015
:106A4000000CBCF1000F0DD1C4E900652C6074602E
:106A50001CE0FFF77DFF013645F10005361845EBD8
:106A6000E070E4E7DCE90420D4E90431934271EBFF
:106A7000000E1DDAD21ADCF8043060EB0100CCE91C
:106A80000420C4E900C31C60CCF804403368B3425E
:106A900009D09C4207D10D4B1C6824B9FFF77EFF3B
:106AA0002146FEF715F887F31188BFF36F8FF8BD05
:106AB0009B1A61EB0001AC45C4E90431C4D0DCF899
:106AC00000C0BEE7C0060020E8010020D819002061
:106AD0002DE9F84FEFF3118C202383F31288BFF3D5
:106AE0006F8FDFF8B0A0DFF8B0902C4FC9F800002E
:106AF000DAF800000024504508BF00200025D7E93F
:106B00000021D9F80030E04678B3D0E9046C4FEAB0
:106B1000E37EB3427EEB0C0B05DAF61A6CEB0E0447
:106B2000C0E9046421E0B21841EBE671C0E9044514
:106B3000C7E90021FFF716FF88F31188BFF36F8FB5
:106B400083689847EFF31188202383F31288BFF3FB
:106B50006F8FD9F80030DAF800009B1B5045C4460F
:106B6000C9F80030CBD1D7E900219A1841EBE37383
:106B70000024C7E90023C9F80040FFF70FFF2146B2
:106B8000FDF7A6FF88F31188BFF36F8FBDE8F84FBC
:106B9000FFF794BEE8010020D8190020C0060020AD
:106BA00010B5EFF31184202383F31288BFF36F8FA6
:106BB000FFF7CEFE054A0346D2E90001181841EB63
:106BC000E37184F31188BFF36F8F10BDC0060020FE
:106BD00073B506460D4601F063FF78B90B4B9B6811
:106BE000DC6E7CB12A1D09D200200021CDE9000114
:106BF00046F00401204602F0DFF808B9002401E065
:106C00000460041D204602B070BD00BFA41900201E
:106C100038B5064C064DAC4201D3002038BDD4E94E
:106C20000112204602F0C0F81434F4E77802002084
:106C3000780200201FB5094A92E8030002AB83E8FE
:106C400003004FF480620093054906484FF0FF337C
:106C5000FFF726FA002005B05DF804FBF091000074
:106C600080320020C806002010B50A4C23681BB1F2
:106C700001232360002010BD00F0EAF80028F7D0BF
:106C80000138062803D8044B53F8200010BD0348F0
:106C900010BD00BFDC190020D8930000FE8FFFFF5D
:106CA000BFF34F8F0549064BCA6802F4E0621343F5
:106CB000CB60BFF34F8F00BFFDE700BF00ED00E0EA
:106CC0000400FA0510B4094B09490A4C4FF0FE3292
:106CD000C3F800244968C3F80424C3F80824C3F89F
:106CE0000C240023C4F8003510BC084700B0025043
:106CF000F001002000A00250D0E90012014BC3E9CE
:106D000000127047F001002010B5044650B16368CE
:106D100013F0685F05D0064A934202D00023236037
:106D2000626010BD034B04485B689847EFE700BF03
:106D30002C5F5CA9F0010020F4930000C8B1436807
:106D40000D4A934213D013F0685F0ED0012350E830
:106D5000002F194640E8001C9CF0000FF7D1012AD3
:106D6000F5D0BFF35F8F0020704704487047044898
:106D700070476FF4E04070472C5F5CA9E98FFFFF1C
:106D8000EA8FFFFF80B14368094A93420AD013F0AB
:106D9000685F05D0BFF35F8F00230360184670471C
:106DA00004487047044870476FF4E040704700BFE4
:106DB0002C5F5CA9E98FFFFFEA8FFFFF10B5044647
:106DC00020B1044B63600022226010BD0248FFF72F
:106DD00079FFF6E73A00003A1C94000070B5D0E95C
:106DE0000023174C174D6360D0E90230C4E902302C
:106DF00022604868D1F800C0134BC3E900C0D5F841
:106E00001801D1F808C0C3F808C010F0685FD1F8C5
:106E10000CC00969C3F80CC0196110D00B49C5F842
:106E2000BC110023C5E9453105F58A70C5F8B831B4
:106E30009047236805F5DC70BDE87040184770BDC9
:106E40000C020020F4190020F80100202C5F5CA93E
:106E500038B500F02FF820B1032400F063F8204685
:106E600038BD00F031F898B900F0ACF898B90F4D82
:106E7000D5F828391B0EF02B08D1D5F8242A0C4B55
:106E80009A420AD0072400F017F8E6E70624FAE74A
:106E90000424204638BD0024F5E7012000F092F8D4
:106EA00004460028F7D1C5F80C0AD8E700B0025014
:106EB0000000E0200020704700207047014BC3F81D
:106EC000040A704700B0025010B5114800F048F8AD
:106ED00000B110BD0F4800F043F80028F9D10E4C66
:106EE000204600F03DF80028F3D10C4B0C481C6004
:106EF00000F036F801460028EBD100F02DF80446EA
:106F000008B1204610BD00F03FF82046FAE700BF68
:106F10004C02002048020020440200203C020020D5
:106F20004002002008B5084800F024F8074800F0A7
:106F300021F8074800F01EF8064800F01BF8BDE8ED
:106F4000084000F00BB800BF4C02002048020020AF
:106F5000440200204002002000207047704700BF1C
:106F600008B5034B02681B6810689847002008BDED
:106F70000C02002008B5034B02685B681068984754
:106F8000002008BD0C02002070B5094C094D206995
:106F9000AB68984718B1084B08485B689847084A9F
:106FA000EB68206900211160BDE87040184700BF00
:106FB000F80100200C020020F001002040940000A5
:106FC000F0190020F8B51A4D1A4E0446B268286927
:106FD0009047E8B9184F3B684CB1A3B1012B19D0C9
:106FE000013B3B602869F36898470020F8BD43B92E
:106FF000124A0121C2F800151149D1F81029002ABE
:10700000FBD101333B60F368286998470020F8BD45
:107010000C48F8BD0A4AD2F81039002BFBD1074AB8
:107020006FF07E40C2F80035FFF748FF3B68D7E7B6
:10703000F80100200C020020F019002000A00250EE
:1070400000B00250E98FFFFF0FB407B5064B04AA4A
:10705000186852F8041B019200F008F803B05DF8BC
:1070600004EB04B0704700BFA49200002DE9F04F7C
:107070008DB043680293837815469A07804640F1A5
:107080000D8100240E78002E00F00A81252E0BD0F1
:107090004B1C03930134029B41463046984700281D
:1070A000C0F2F6800399EDE74E788B1C252E0393F2
:1070B000F0D00027B946BB46BBF11F0F38D8A6F168
:1070C0002003102B0AD8DFE803F02A090930090948
:1070D000092109090928092D09091F00A6F1300312
:1070E000092B33D92A2E37D11BF0400F55F8043B1A
:1070F00040F08280002BA7BF4BF0200B9946C3F1D4
:1071000000094BF0280B01E04BF0010B039B13F837
:10711000016B0393002ECFD130E04BF0020B4BF00C
:10712000040BF3E74BF0080BF0E74BF0100BEDE727
:10713000BBF17F0F19D8A6F13003092BD2D81BF071
:10714000400F03D00A2101FB0737DFE70A2101FBCB
:1071500009394BF0200BD9E72E2E06D11BF0400F3A
:1071600040F09E804BF0400BD0E76C2E31D02BD8F6
:10717000682E36D06A2E3CD04C2E3AD0002F46F0E6
:107180002003B8BF2BF04002A3F16501BCBF1FFA7A
:1071900082FB0027022901D9612B2FD1073525F069
:1071A0000705DFF8ACA2083507271BF0080F66D0EB
:1071B0000AEB070B56465E4563D1A4EB0A0A06EBC1
:1071C0000A02A9EB07096FE1742E9FD07A2E9DD099
:1071D000D4E71BF0800F18BF4BF4007B4BF0800B03
:1071E00094E71BF4807F18BF4BF4007B4BF4807B4B
:1071F0008CE74BF4207B89E71F4687E7A6F1630104
:10720000122900F2F080DFE811F013004F00EE00C9
:10721000EE00EE00EE004F00EE00EE00EE00EE009D
:10722000EE00FE00E900EE00EE001B00EE00AF00F5
:1072300055F8043B8DF8183001270DF1180AB4E712
:1072400055F804AB834BBAF1000F08BF9A461BF008
:10725000400F14BF39464FF0FF31504601F01FFE7A
:107260000746A2E7029B41462020984700280FDBF3
:10727000013EB742F6D34C44A41BB14698E74E46B4
:10728000F7E716F8010B029B41469847002892DA6F
:1072900098F8023043F0040388F802304FF0FF34CE
:1072A00020460DB0BDE8F08F1BF0800F34D01BF4EA
:1072B000007F2CD0073525F00705AA4669685AF8E3
:1072C000080B2BF010050029ADB237DA404261EB14
:1072D000410145F480650DF1180B0A235A4601F06F
:1072E000EAFDA0EB0B0301936B0662D5019B25F031
:1072F00001019F4289B240F3A180002E00F09980E5
:1073000015F0100240F09C80BB460D4623E0AA46D3
:107310005AF8040BC117D4E7AA461BF4807F5AF829
:10732000041B01D10846F5E71BF4007F15BF48B2E6
:1073300008B241F3C01141F3C031C2E750EA010382
:10734000C9D11BF0400FC6D0002FC4D12BF01102C1
:1073500095B2BB46019740F2064115EA01021CBFF7
:107360000BF1010B00222CE02BF010021FFA82FB24
:107370000A231BF0800C49D01BF400711DBF073598
:1073800025F00705AA46AA461ABF5AF8080B6968ED
:107390005AF8040B50EA010545D12BF016051BF0F5
:1073A000400FADB242D0002F40D12BF0170295B262
:1073B000019715F0100248D0019B002E42D103F135
:1073C000010B29075AD4EB0706D5D9456FDD019982
:1073D000A9EB0B035F18CB465B4649E04BF0100B63
:1073E00010237826C5E7782B04D1C6F1780343F043
:1073F0001003BEE7029B4146252098470028FFF670
:1074000047AF023447E608230026B2E7AA461BF43A
:1074100080715AF8040BBDD01BF400711ABFC0B2C2
:10742000614680B2B6E72BF0060295B20DF1180B5B
:1074300054E725F01105ADB2BB468CE70D46B8E721
:107440003B460D4603F1020BBBE7DDF804B082E7D3
:10745000F7950000F0950000CDE904324146029B0B
:10746000202098470028FFF613AF049B059A0133AC
:107470009945F1DCA4EB0B01CC189B460AB3029BA7
:107480004146302098470028FFF602AF8EB90134FC
:107490002744019B391B994224DC1D465DBB019AA0
:1074A000A9EB0B09224455461446914435E0019F4F
:1074B00092E7023441463046029B98470028E7DABB
:1074C000E6E640F206410D42E2D015F0020F14BF8D
:1074D0002B20202015F4806F04F10104414618BFD1
:1074E0002D20E9E7029B414630209847002804F10F
:1074F0000104CEDACCE606AB013D4146585D029B65
:1075000098470028CADAC3E6029B414620209847E4
:10751000002804F10104FFF6BBAEA9EB0403002B25
:10752000F2DCBFE57047836800EBC101B3F5004FA3
:107530002CBF51F8220031F81200704700EBC10156
:107540008068B0F5004F2CBF41F8223021F812308E
:10755000704708B50122FFF7E6FFD04008BD8368F9
:10756000B3F5004F00EBC10108D34B681AB143F0EB
:1075700001034B60704723F00103FAE74B881AB10F
:1075800043F001034B80704723F00103FAE75300F7
:107590000122FFF7D3BF8368B3F5004F34BF042344
:1075A0000823C91A081AC0087047B0F5004F34BF45
:1075B00004230823481C0833A0EBD300B0FA80F062
:1075C000C0F11F0070472DE9F041174603220E4617
:1075D0000446FFF7A8FF8642054607F104080AD1D2
:1075E000E3680122BA4023EA0203E360002344F87F
:1075F0002830BDE8F081314602222046FFF793FF94
:107600002B460646014644F8285020460322FFF741
:1076100095FF3346294620460222BDE8F041FFF798
:107620008DBF70B50D4686680446FFF792FFB6F52C
:10763000004F014601D3012809D03046FFF7B5FFBE
:10764000294602462046BDE87040FFF7BCBF70BD2A
:107650002DE9F04705468068FFF7A7FF05EB800A94
:107660008846DAF810900646B9F1000F1BD00327C0
:10767000DAF8104028462146FFF76BFF404507D354
:10768000324621462846FFF79EFF2046BDE8F08798
:10769000032221462846FFF746FF013FCAF81000A3
:1076A00001D08145E4D1EB6801364FF0FF34B4409E
:1076B0001C40EAD094FAA4F2B2FA82F2131D55F8F3
:1076C0002340DEE72DE9F041144605460E46FFF75C
:1076D00040FFA4EB0608371B0744424631462846C4
:1076E000FFF755FF3A4621462846FFF750FF43462D
:1076F000002221462846FFF721FF21462846FFF7B2
:1077000028FF3B46211800222846BDE8F041FFF73C
:1077100015BF2DE9F041164604460F46FFF719FF45
:10772000314605462046FFF714FF05442A463946F0
:107730002046FFF72CFF31462046FFF70AFF2B4675
:10774000311800222046BDE8F041FFF7F7BE2DE9D1
:10775000F0410D4686680446FFF7FBFEB6F5004F84
:10776000014601D3012832D03046FFF71EFF04EB5B
:1077700080010E6996B9E368012282401343E360F9
:1077800002220D612B4629462046FFF7D7FE032231
:1077900029462046BDE8F041FFF7D0BE022231461F
:1077A0002046FFF7C0FE2946034607462046FFF75E
:1077B000C5FE0322334629462046FFF7BFFE394661
:1077C0002B462046FFF7BAFE02223146E1E7BDE82C
:1077D000F081F8B50C460546FFF7BBFE26180122DE
:1077E00031462846FFF79FFEC3070CD43146284692
:1077F000FFF717FF21462846FFF7ABFE2146221868
:107800002846FFF786FF002221462846FFF78BFE19
:10781000271A012239462846FFF785FE10EA02069C
:1078200013D139462846FFF7FCFE2146324628464A
:10783000FFF779FE2246211A2846FFF76AFF214604
:1078400032462846FFF76FFE241A21462846BDE837
:10785000F840FFF77CBF38B571B105682846FFF7DF
:107860009AFE0022044601462846FFF778FE21468C
:10787000BDE83840FFF7ADBF38BD70B5066809B93F
:10788000002070BDB368B3EBD10FF9D9B3F5004F49
:1078900034BF04230823CC1D1C44E4082146304691
:1078A000FFF7D6FE05460028EAD001463046FFF72E
:1078B00050FEA04209D92C44294630462246FFF703
:1078C00001FF21463046FFF742FF3046012229469C
:1078D000FFF745FEB368B3F5004F34BF0423082318
:1078E00003EBC5031844CCE72DE9F84306681446BA
:1078F000B26801F1FF39B2F5004F34BF0423082309
:1079000019EA01090F460BD0494239408B424F46D4
:1079100028BF0B46894654B900252846BDE8F883A0
:107920009942F8D82146BDE8F843FFF7A6BFB2EB6D
:10793000D40FF1D9E11DB2F5004F394434BF042210
:107940000822C91A1144C9083046FFF781FE804653
:107950000028E1D0B368B3F5004F34BF04230823F7
:1079600009EBC0051D4435447B1E1D44B5FBF7F5EE
:107970007D43A5EB090529463046FFF70CFE2C4454
:10798000073424F00704A41B804507464FEAE404AB
:1079900008D2024641463046FFF794FE4146304643
:1079A000FFF7D5FE39463046FFF7D3FD3844844211
:1079B00008D2394630462246FFF784FE214630463B
:1079C000FFF7C5FE012239463046FFF7C8FDA4E7A0
:1079D000B2F5802F2CBF08230423D21A2DE9F041E1
:1079E0008C18CD1D25F0070524F00704641B002624
:1079F000E40805602146AC60EE602046FFF7D5FD47
:107A0000421D9200013002F107074FEAD707A2F1A9
:107A100010023146B8BF324605F1100001F037FAC6
:107A20003A4631462846FFF7B2FD334632463146E4
:107A30002846FFF783FDA4EB0708284631460122BC
:107A4000FFF78DFD42463946FFF7A1FD3B46324622
:107A500039462846FFF772FD21462846FFF797FD75
:107A60004346324621462846FFF768FD2146284610
:107A70000122FFF774FD3946BDE8F041FFF767BE0C
:107A8000002070470FB407B504A951F8040B019109
:107A9000F8F7EEFC03B05DF804EB04B07047036840
:107AA00000220BB9184670478B4210D10B6842B9BF
:107AB00042680360914200D1436000230B600120C3
:107AC000704713604368994208BF4260F5E71A4661
:107AD0001B68E6E7038B13F0070305D10368002B4F
:107AE0000CBF002003207047022B05D1408BB0FA59
:107AF00080F0400980007047012B05D10368002BFE
:107B00000CBF0020052070470020704710B50C46C0
:107B100000B111B96FF0150010BD081D00F0D2F8CA
:107B20000028F9D1A368032BF6D9F3E72DE9F0413A
:107B30000D4607461946281D90461E4600F0D3F80C
:107B4000044638B13346424629463846A446BDE885
:107B5000F0416047BDE8F08110B4EFF311822024BA
:107B600084F31288BFF36F8F416110BC0121F8F7D5
:107B7000B1BC38B50C46054658B151B10B6843B19C
:107B80004B6833B11C22002101F081F92C610020E7
:107B900038BD6FF01500FBE770B505460E46FFF7E0
:107BA000B5FF041E14DBEFF31182202383F3128848
:107BB000BFF36F8F6B8B2C8B4FF6FF718B4204F0F2
:107BC000070407D182F31188BFF36F8F6FF00A04A7
:107BD000204670BD022C0CD101336B8382F31188D7
:107BE000BFF36F8F0023224631462846FFF79EFFE2
:107BF000EEE7062C14D8DFE804F004131313041A7C
:107C00000400002333606B683BB9C5E90066ACB97A
:107C100002212846F8F75EFCDAE71E606E60F6E7A0
:107C200082F31188BFF36F8F6FF00404D0E782F303
:107C30001188BFF36F8F6FF08504C9E782F3118855
:107C4000BFF36F8FC4E710B5EFF31182202383F3E6
:107C50001288BFF36F8F048B04F00704022C0AD044
:107C6000012C0CBF6FF004006FF0850082F31188C7
:107C7000BFF36F8F08E0438B013B9BB2438323B973
:107C80002146F8F727FC204610BD2046EEE738B520
:107C9000A8B1A1B1EFF31185202282F31288BFF3BE
:107CA0006F8F048BFFF7FBFE30B104F0070085F304
:107CB0001188BFF36F8F38BD6FF07700F7E76FF073
:107CC0001500F8E7034658B1426802F00302012AA2
:107CD00003D0032A04D1026812B1002098607047D3
:107CE0006FF0150070474268816002F00302032ABA
:107CF0004FF0000203460CBF006810465A60704700
:107D0000F0B5C6684568C369AF1B04464069BB420D
:107D100098BFFF1AA5EB0000944698BFF6181A1AF0
:107D2000D81B2368AD1B62452B4428BF62460B60FD
:107D30006368904228BF104603446360F0BDD0E9F9
:107D40000123D21A8A420CD31944C368C269C0E91C
:107D50000111C91A8A4201D9002070471344C36037
:107D6000FAE76FF0150070472DE9F34180460E46A3
:107D7000154600272A4601A94046FFF7C1FF3146B4
:107D800004460246019801F074F82D1B274426444E
:107D900001D0002CEED139464046FFF7D0FF3846DF
:107DA00002B0BDE8F081F0B5044686690569C06996
:107DB000A368AF1BB842944698BF3618A3EB0502E0
:107DC0002368A5EB060598BF3F1A2B446245A0EB3C
:107DD000070028BF62460B602369904228BF104607
:107DE00003442361F0BDD0E90423D21A8A420CD3A4
:107DF0001944D0E90632C0E90411C91A8A4201D9EE
:107E00000020704713448361FAE76FF01500704754
:107E10002DE9F34180460D4616460027324601A95A
:107E20004046FFF7C0FF04462DB10246019928469F
:107E300001F01FF82544361B274401D0002CEDD15A
:107E400039464046FFF7CFFF384602B0BDE8F08123
:107E5000704710F0700F08D100F07F0310F0800F12
:107E600018BF1033012098407047002070472DE95B
:107E7000F84306460F469046994604254B4642462F
:107E800039463046FAF7AAFF10F10B0F044603D12A
:107E9000FEF7E8FB013DF1D12046BDE8F883002064
:107EA000F8F7ACBF006840B150F8043C5B688B4207
:107EB000A0F1040001D04068F5E77047006850B1B8
:107EC00050F8043C5B685B689B788B42A0F104002F
:107ED00001D04068F3E7704730B5006888B150F8CA
:107EE000043C5B681A6A1D7F04380023043ADCB244
:107EF000A54201D84068F1E7013312F833408C42C3
:107F0000F5D130BD08B5F9F74DF928B1406810F149
:107F1000100F14BF0020012008BD4B1CDBB2817084
:107F2000817680F82530C37600F8061C704750E94A
:107F30000231D0F89C0018470369002283F84A20D8
:107F40007047036993F84A0048B193F8480030B18C
:107F5000D3F8902053685169D0695B1AC01A7047F2
:107F60000369002283F84B207047036993F84900A6
:107F70007047036993F8482012B193F84A202AB950
:107F800093F8490018B193F84B00704701207047EF
:107F9000012070470369C3E90012704770B5046996
:107FA0000546D4F88C00FFF733FFD4F88C301A69FB
:107FB0009968914204BF002284F8492094F8A020D7
:107FC00006469AB15A685969DB69521A9B1A3F2BC7
:107FD0000CD994F89E3033B16B681B6A2246187B2B
:107FE0000021F9F7C9FB002384F8A030304670BDAA
:107FF00008B50122FFF7D2FF013818BF4FF0FF305C
:1080000008BDFEE7012801D1EFF30583FDF79ABC17
:1080100001460068FFF7F6BF08B5F9F73DFDBDE87A
:108020000840F9F75DBD00210120FFF7EBBF61B605
:1080300062B680F31188BFF36F8F704772B600236A
:1080400083F31188BFF36F8FBFF34F8F30BF62B6DA
:10805000BFF36F8F704772B6002383F31188BFF3AD
:108060006F8FBFF34F8F20BF80F31188BFF36F8FE7
:1080700062B67047202809D9B0F1004F08D80138FE
:10808000B0FA80F0C0F11F00400070470820704730
:108090003E20704708B5FAF7ADF9002008BD10B5CD
:1080A0000369C0E905330023C360837F044613B12D
:1080B000407AFBF741FD0123237700236377E377C1
:1080C000A37710BDFDF7C0BDFDF736BE037802797A
:1080D00003F00F011AB959B14FF0FF30704708296A
:1080E000FAD8012A04D183F0080040F3C000704799
:1080F00043F3C000704738B50446FAF70BFA05465B
:1081000060B1037A6BB120460024FBF799FD284645
:10811000AC77FFF7C4FF2C72204638BD6FF0150016
:10812000FBE76FF07700F8E770B504460E4615469A
:10813000FAF7D0FE30B906B925B12046BDE8704047
:10814000FAF710BF70BDC343C3F3C01300F00F00B4
:1081500000EB0310704708B5FAF786FF818208BD6F
:1081600008B5FAF781FFEFF31183202282F312881A
:10817000BFF36F8F02690A60027B2AB9807D83F3A7
:108180001188BFF36F8F08BD0420F8E70369C9B2F7
:108190000C2201FB0233186C00F00700704770B529
:1081A000C9B20369EFF31185202484F31288BFF369
:1081B0006F8F0C2606FB0134246C14F0C00408D029
:1081C000A24206D085F31188BFF36F8F4FF0FF30C6
:1081D00070BD06FB013301221A6485F31188BFF3D9
:1081E0006F8F436803EBC1035B6898470020EFE79C
:1081F0008022FFF7D4BFF8B5069F0469C9B2EFF338
:108200001186202585F31288BFF36F8F0C2505FB9F
:108210000144256C05F0070CBCF1010F0CD127645B
:1082200086F31188BFF36F8FC4E90E23436853F8B8
:10823000313098470020F8BD05F0C005AF4286F305
:108240001188BFF36F8F0CBF6FF077004FF0FF30D6
:10825000F1E713B580240094FFF7CDFF02B010BD05
:1082600010B40069CBB21C2403FB0400002110BC35
:1082700010470020FCF748BE002000F0E3B910468C
:10828000FDF7C8BD43685B68D3F810350B6000206C
:10829000704743685B6802EA010021EA0201C3F803
:1082A0000805C3F80C150020704743685B68002080
:1082B000C3F80815704743685B680020C3F80C15C5
:1082C000704743685A68D2F8043521EA03000B402E
:1082D000C2F80805C2F80C350020704710B50369D4
:1082E0005868F8B1884219D19C6808685860A14262
:1082F00000D19860002008602AB15A680A609A6824
:10830000596002B99960002010E0814206D10868E6
:10831000206098688142EDD19C60EBE704460068DC
:108320000028F2D1002AE8D16FF0150010BD13B576
:108330004FF080520829136E526E28BF082112BADE
:1083400000921BBA0C460A466946019300F091FD63
:10835000204602B010BD30B543681360057A44680A
:1083600004EBC504A34202D36FF0010030BD5C7979
:108370008C4201D00833F0E70020F7E743681B6820
:10838000D3F88004C3F88004704742681368D3F8B8
:10839000100150B1D269002012780A70C3F81001A0
:1083A000D3F8102101221A6070474FF0FF30704758
:1083B000002A0FDD42681368D3F8100158B100207D
:1083C000C3F81001D269D3F8100112780A700120A5
:1083D000186070470020704710B54368196803693A
:1083E000EFF31182202080F31288BFF36F8F18689B
:1083F000002484731B680120D8734FF48003C1F8F4
:10840000043382F31188BFF36F8F10BD03691A68BC
:10841000012191731B680022DA73704702691168A9
:108420000346C87B40B15B681B68D3F8580118B19C
:1084300000230B6113689889704743681B68D3F861
:108440001001003818BF0120704743681B681022D4
:10845000C3F80423704743681B681022C3F808233D
:10846000704743681B684FF40072C3F804237047D9
:1084700043681B684FF40072C3F80823704738B58F
:1084800043681D68D5F804335B02044605D4D5F86B
:10849000040310F0100006D138BDFFF7BFFF00281D
:1084A000F5D00120F8E72046FFF7C7FF003818BFD6
:1084B0000120F1E7012070470369186801601B681B
:1084C0005A60704702680346D2F8580140B95B68A9
:1084D000DB0706D4D2F82001003818BF012070470E
:1084E0000120704710B4436802691B68D3F8041375
:1084F000C90517D5D3F82011A1B1EFF311812024BC
:1085000084F31288BFF36F8FD3F8204134B1002475
:10851000C3F82041D3F820410124DC6081F31188A5
:10852000BFF36F8F1468D3F858115CB161B10021AB
:1085300021611468A47B3CB14FF48000C3F80803A8
:108540001368997310BC7047D3F8241121B100212E
:10855000C3F82411D3F8243112681368002BF1D02A
:10856000516810BC18472DE9F041066933689C89B1
:10857000BFF35B8F94420546A8BF14461033012712
:1085800053E8002F002A03D143E800700028F7D1F8
:10859000BFF35B8F0CBF3B4600232BD133682246D1
:1085A000986800F066FCEFF31188202383F31288AB
:1085B000BFF36F8F69680846FFF784FF326840B9E0
:1085C0001061044688F31188BFF36F8F2046BDE821
:1085D000F0810B689268C3F844250022C3F848452F
:1085E000C3F82021D3F82011C3F85821D3F858211B
:1085F0009F60E7E71C46E9E700F150039B009BB250
:1086000003F1804303F5883300221A601B6870472A
:10861000FEF72ABB08B5F9F753F9F9F727FABDE8D1
:108620000840FEF721BB004700F0AFB8C00000F1E2
:10863000804000F5F830C0F81015C0F814257047D8
:10864000FDF77AB9FCF7D6BBF7B5019001A8DDE9D3
:10865000084716461D46FCF7DFFC019BB6F1000CEF
:1086600018BF4FF0010C00EB83000B1E18BF012355
:10867000002D43EA4C0314BF4FF00C0C4FF0000CDC
:10868000002C43EA0C0314BF4FF4E06C4FF0000CD5
:10869000002F43EA0C03D0F8002714BF4FF4403CEE
:1086A0004FF0000C43EA0C0322EA030301B10978FE
:1086B0000EB13678760019430DB12D78AD003143F7
:1086C0000CB12478240229430FB13F783F040C43B6
:1086D0003C43C0F8004703B0F0BD1FB50DF10F03D8
:1086E000019300238DF80F1000931A461946FFF7E7
:1086F000ABFF05B05DF804FB38B5054608460C46EF
:10870000FCF7DCFCB0B10846FCF7CCFC90B908469D
:10871000FCF7BCFC2A6801238340C2F808332A68AE
:1087200003B202EB8303D3F8102522F00302C3F84F
:10873000102538BD20460021BDE83840FFF7CDBFE9
:10874000FCF742BDFFF7D8BF00F180431A68002A4A
:108750001FBF00221A601B68012008BF002070475D
:108760004FF080434FF46072C3F8042370474FF01A
:1087700080434FF46072C3F80823704708B5FDF7D3
:108780008BF8BDE80840FCF713BC08B1F9F77ABED6
:108790007047704740B1C368587810F001001EBFA1
:1087A0001878B0FA80F040097047EFF31183202366
:1087B00083F31288BFF36F8FFEE708B5FFF7F5FF6D
:1087C00010B5D0E9003433B90020E268537843F0A3
:1087D0000103537010BD204698470028F4D00028AC
:1087E000B8BF4042E368FF28A8BFFF201870ECE73D
:1087F00000F04DBB00F03DBB70474169836843EA20
:10880000010212F003020FD1C2600269013A01FBBA
:10881000023382689A4201D900207047C2681A6008
:108820004269C3609B1AF4E76FF01500704710B5FA
:10883000C0E904320023816083610446FFF7DDFF55
:108840000028A8BFC4E9004410BDF8B504460D4691
:10885000EFF31186202383F31288BFF36F8FC7686D
:108860006FB900F0C1F950B18767456100F05DF95B
:10887000314604F10800BDE8F840FDF773BEE36837
:108880002B60A369E560013BA36186F31188BFF308
:108890006F8FF8BD08B52024EFF3118384F312889D
:1088A000BFF36F8FFFF7CAFBF6E790F90E308B42EC
:1088B00001D0FDF713BE0020704703460020C3E936
:1088C0000200C3E9003370472DE9F8439946044696
:1088D0009DF820300D46904600F10806EFF3118711
:1088E000202282F31288BFF36F8F03B145683046B0
:1088F00000F07AF958B100238367C0F8148000F0C3
:1089000014F930463946FDF72DFE00200CE0B9F190
:10891000000F1CD00821FEF75BF938B987F31188E6
:10892000BFF36F8F6FF00B00BDE8F8830122C0F832
:1089300004800260016801F0030165B922680A43FE
:10894000026062682060002ADBD16060D9E7C8F865
:1089500000904046EEE72A68032A0BD80160616860
:1089600011B9C4E90000CCE70A6802F0030202432F
:108970000A60EAE722F003020A4302602A6802F072
:10898000030240EA02032B60BBE710B5044630B196
:108990000268930703D0446809B100F0FEF920464D
:1089A00010BD07B50123009300230A461946FFF7BF
:1089B0008BFF03B05DF804FB3AB18A4205D3C0E9EE
:1089C0000212C0E90000002070476FF015007047E8
:1089D000026801238B4022EA0303036022FA01F0BC
:1089E00000F00100704720B100221146883000F0ED
:1089F00054B9704773B50446EFF31185202383F310
:108A00001288BFF36F8F0023A0F1100603210438F2
:108A10000193FFF7DDFF28B1A369019301A9304657
:108A2000FDF7E4FA85F31188BFF36F8F02B070BDD4
:108A300038B504460D461022002100F028FA656082
:108A400038BD13B501900846EFF31184202383F35A
:108A50001288BFF36F8F01A9FDF7C8FA84F311885C
:108A6000BFF36F8F02B010BD10B5FFF7EAFF041E11
:108A700008DDEFF31180202383F31288BFF36F8F9B
:108A8000FDF7A0FD204610BD38B5302204460D4646
:108A9000002100F0FCF94FF480736560E36038BD9D
:108AA000EFF30580003818BF012070476FF05700C2
:108AB0007047FDF769BDD0E9003213605A600023AA
:108AC000C0E90033704708B5FFF7F5FF437B23F09B
:108AD000020343730023836008BD38B504460D4686
:108AE000FDF7DCFB637B43F002036373E5B1A56034
:108AF0002B689D4209D16B68C4E900531C606C600F
:108B000012E06A689A42F6D01B68002BF3D094F901
:108B10000E2093F90E108A42F3D09142F1DD5A688B
:108B2000C4E9003214605C6038BD10B5EFF3118405
:108B3000202383F31288BFF36F8FFDF7C7FB84F305
:108B40001188BFF36F8F10BD10B50446183000F0C8
:108B5000C6F8EFF31181202383F31288BFF36F8FE0
:108B6000627B12F0100204D081F31188BFF36F8F83
:108B700010BD2046BDE81040FDF7DCBB08B5EFF3A3
:108B80001181202282F31288BFF36F8F83680BB1AB
:108B9000FFF799FF81F31188BFF36F8F08BD38B5D8
:108BA0000446EFF31185202383F31288BFF36F8F00
:108BB000437B13F0280F0BD183680BB1FFF783FFC2
:108BC000637B51B903F0FB0363732046FDF77EFB23
:108BD00085F31188BFF36F8F38BD03F0EB03F3E724
:108BE00001211838FFF7DBBF38B5EFF311852023DB
:108BF00083F31288BFF36F8F0468A0420DD034B1A5
:108C00002046FFF760FF04F1180000F068F885F3D4
:108C10001188BFF36F8F204638BD0024F7E710B5E9
:108C2000FFF7ACFFBDE81040183000F058B838B579
:108C300004680546AC424FF0000000D138BD002C5E
:108C4000FCD02046FFF7EBFF2046FFF76EFF2C68B5
:108C50000120A542F1E7EFF31181202282F312886F
:108C6000BFF36F8F027BD2070CD581F31188BFF35E
:108C70006F8F002383F31188BFF36F8F042318468F
:108C800002DF7047437B1B0704D581F31188BFF3D4
:108C90006F8F70470122FDF74DBB38B5EFF311859B
:108CA000202383F31288BFF36F8F0468A04212D091
:108CB0009CB1A16762612046FFF705FF04F118002F
:108CC00000F00DF82046FDF701FB012085F3118827
:108CD000BFF36F8F38BD0020F8E72046F6E710B5E8
:108CE000EFF31184202282F31288BFF36F8F0368A1
:108CF0003BB1FDF737FE002084F31188BFF36F8F7F
:108D000010BD6FF01500F7E708B5FDF749FF08BD86
:108D1000B3F1FF3F08BFB2F1FF3F70B504461D46F7
:108D2000164613D01A4315D06FF00102921B4FF074
:108D3000FF3363EB0501002904DAFDF731FF8219E7
:108D400041EB0501C4E90021204670BD4FF0FF3220
:108D50001146F7E70022FBE7B3F1FF3F08BFB2F18E
:108D6000FF3FF8B5074616461C4610D054EA0203EA
:108D700011D0FDF715FFB0420A46A14103460AD2C1
:108D8000F31A64EB0204C7E900343846F8BD4FF02B
:108D9000FF331C46F7E70023FBE720B1011F50F823
:108DA000040C00F04AB8704710B400F10C04C0E99C
:108DB000034410BCFEF70CBE2DE9F04F89B0DDE98D
:108DC000126705463B46914606A832460591FFF7D5
:108DD0009FFFDDE9063405F1140ACDE90234EFF313
:108DE00011844FF0200888F31288BFF36F8F05F1CC
:108DF0000C0B05994A462846FEF776FD30B184F300
:108E00001188BFF36F8F09B0BDE8F08F3E43F6D0F5
:108E1000DDE9022306A8FFF79FFFDDE906675A4652
:108E2000CDE9006721465046FDF72CFBEFF3118496
:108E300088F31288BFF36F8FDBE738B50446EFF392
:108E40001185202383F31288BFF36F8FFEF703FD94
:108E500004F10C00FFF7EBFE30B1294604F11400D9
:108E6000BDE83840FDF77EBB85F31188BFF36F8FF7
:108E700038BD0A44914200F1FF3300D1704710B56C
:108E800011F8014B03F8014F9142F9D110BD024492
:108E90000346934200D1704703F8011BF9E710B570
:108EA000024601448A42134603D01C780132002C4A
:108EB000F8D1181A10BDF0B5C3F137070446FFB258
:108EC00003F01F031046082BE6B233D0102B3ED020
:108ED0006508A40844EA817445EAC1752D194FEA72
:108EE000910242EB5102290941EA02716D1842EBED
:108EF0001212290A41EA02616D1842EB1222290C72
:108F000041EA02416D1842EB1242AD1842F10002F3
:108F1000EC0844EA4274D10804EB8402A6EB420553
:108F2000EDB2092D0CD90134A5F10A0541F100017A
:108F3000EDB212E0E40844EA417406F00705C908FE
:108F4000303554EA010200F8015BBCD1F0BD2409C0
:108F500044EA017406F00F050909092D84BFED19D3
:108F6000EDB2EDE70148006870470000580E0020A0
:108F7000C471FF7F010000004124000000000000D8
:108F8000D93D000008900000C95B0000000000000F
:108F9000116C000000000000A14100001C900000C6
:108FA000A141000030900000992400000000000062
:108FB00011860000000000000546000058900000E7
:108FC000C116000044900000514000000000000065
:108FD0006D490000000000001D240000000000009A
:108FE000711800000000000015860000000000005D
:108FF000356C000000000000A1250000000000000A
:109000009F7E0000000000007D950000B8920000E7
:10901000C892000052020020181900208C95000010
:10902000E492000014930000540200206C19002008
:109030009A950000FC920000149300005602002054
:109040007819002087940000A003002008920000F7
:109050005002002000000020B0950000389300006E
:109060007C930000580200203C0100207D87000016
:1090700027860000000000002780000058900000B4
:10908000E5840000000000002780000000000000D0
:109090002780000000000000278000003D560000EF
:1090A000278600000000000027800000000000006C
:1090B0002780000000000000278000000000000062
:1090C0002780000000000000278000000000000052
:1090D0002780000000000000278000000000000042
:1090E0002780000000000000278000000000000032
:1090F0002780000000000000FD4900000000000083
:109100002780000000000000278000000000000011
:109110002780000000000000278000000000000001
:1091200027800000000000002780000000000000F1
:1091300027800000000000002780000000000000E1
:1091400027800000000000002780000000000000D1
:1091500027800000000000002780000000000000C1
:1091600027800000000000002780000000000000B1
:1091700027800000000000002780000000000000A1
:109180002780000000000000278000000000000091
:109190002780000000000000278000000000000081
:1091A000278000009D34000027860000000000009A
:1091B0002780000000000000278000000000000061
:1091C0002780000000000000278000000000000051
:1091D0002780000000000000278000000000000041
:0C91E00027800000000000002780000035
:1091F000E79500000001000000C201000000080027
:109200000338FDD870470000F17F00000917000007
:1092100000000000D11500009D7F00005D150000DA
:10922000397F0000437F00003D150000617F000092
:10923000000000006B7F0000000000000000000044
:10924000737F0000917F0000957F00000000000008
:1092500003800000240100201C01002014010020D4
:10926000000000000C010020D9190000CD180000FA
:1092700021190000811900000000002000000000FA
:1092800000000B06020000008C92000000000000AD
:109290005395000026000207000000205B950000A7
:1092A00022000B112C01002019270000613D000055
:1092B000313D000000000000B13E0000A53D00006F
:1092C0007382000079820000313E0000F1810000CD
:1092D00053820000000000008D81000000000000AB
:1092E00000000000FFFF000000030050000000002D
:1092F000010000000060004000000000FFFFFFFFD1
:10930000000000500000000000000000006000406D
:1093100000000000354200008582000093820000BA
:10932000AB820000B7820000C3820000A1400000B1
:10933000DD8200000000000000200040010000006D
:1093400000000000589300000000D601000000005B
:10935000CF1B0020CE1B00200020004064930000A3
:10936000010000006C9300000400000014000000E5
:109370001100000218060001160600038B8300008E
:10938000514500007D83000067850000B183000027
:10939000D98300000D8400001D8400004B84000070
:1093A000578400001D8400003B840000638400009B
:1093B000718400007F840000B5840000B98400003F
:1093C000788F0000788F0000D08F0000D88F0000C9
:1093D0000890000008900000FF8FFFFFFF8FFFFF45
:1093E000FE8FFFFFFE8FFFFFFD8FFFFFFC8FFFFF54
:1093F000FC8FFFFF6D757465785F6672656520632D
:10940000616C6C65642077697468204E554C4C2003
:10941000706172616D6574657200000043616E2752
:109420007420696E697469616C697A65206D757400
:1094300065782C20776173204E554C4C0D0A000046
:10944000436F756C64206E6F74206C6F636B20705B
:109450006F7765722073617665206D75746578002D
:109460004F4E004F4646004C45442073746174656E
:109470003A2025730A0030313233343536373839E3
:10948000414243444546006364635F61636D5F75B9
:1094900061727400757362776F726B71002A2A2A89
:1094A00020426F6F74696E67206E524620436F6E64
:1094B0006E6563742053444B2076322E392E302D46
:1094C000373738376232363439383430202A2A2A4E
:1094D0000A002A2A2A205573696E67205A65706827
:1094E0007972204F532076332E372E39392D31663D
:1094F00038663364633239313432202A2A2A0A002A
:109500006D757465785F696E69742063616C6C65F4
:10951000642077697468204E554C4C2070617261EC
:109520006D6574657200436F756C64206E6F742096
:10953000616C6C6F63617465206D75746578206211
:1095400065666F726520696E697469616C697A69B4
:109550006E6700464C4153485F30005352414D5FA7
:109560003000000001000000757362645F776F7265
:109570006B710001000203000101010101636C6FC6
:10958000636B403430303030303030006770696F9A
:10959000403530303030333030006770696F4035DF
:1095A000303030303030300000010203040506074F
:1095B0007561727440343030303230303000000029
:1095C00000000001010000000000002030303030B9
:1095D00030303030303030303030000100000100A9
:1095E00000006D61696E00737973776F726B710043
:1095F000286E756C6C29002A666C6F61742A0000F5
:10960000000000000000000000000000000000005A
:10961000000000000000000000000000000000004A
:10962000000000000000000000000000000000003A
:10963000000000000000000000000000000000002A
:10964000000000000000000000000000000000001A
:10965000000000000000000000000000000000000A
:1096600000000000000000000000000000000000FA
:1096700000000000000000000000000000000000EA
:10968000000000000000000000000000D4000020E6
:10969000B400002000C2010000000800000000002B
:1096A00000000000000000000000000000000000BA
:1096B000817A000040390020000000000000000016
:1096C000000000000000000000000000000000009A
:1096D00000040000403D00200000000000000000E9
:1096E000000000000000000000000000000000007A
:1096F000000400002515000080000000D1120000C9
:1097000000000000D1120000800000008C02002048
:109710003A000000A00200203A0000007802002079
:109720003A000000B40200203A00000000000000EF
:109730009580000000000000000000004C010020A7
:109740000000000000000000000000000000000019
:1097500000000000D01B00202000000000000000DE
:1097600000000000000000000000000000000000F9
:1097700000000000000000000000000000000000E9
:1097800000000000000000000000000000000000D9
:1097900000000000000000000000000000000000C9
:1097A00000000000000000000000000000000000B9
:1097B00000000000000000000000000000000000A9
:1097C0000000000000000000000000000000000099
:1097D00008000000FF00000000000000030000007F
:1097E00000000000FFFF0F00E8010020E80100205A
:1097F00000000000A16C0000340200202C020020B8
:1098000024020020000000001C020020BD6D0000AA
:10981000096D00003D6D0000856D0000E01900201D
:109820003A00003AE41900203A00003AE819002012
:109830003A00003AEC1900203A00003A44020020B5
:109840000802002000020020FC010020F801002096
:0A985000000000000000000000000E
:10985C005C0200205C020020C036002000000000EA
:10986C00200000001400000000000000780200201E
:10987C007802002000000000000000000E00000034
:10988C008C0200208C020020000000000000000070
:10989C000E000000A0020020A0020020000000002A
:1098AC00000000000E000000B4020020B4020020F2
:1098BC0000000000000000000E000000C8020020A4
:1098CC00C802002000000000000000000E00000094
:1098DC00DC020020DC02002001000000010000007E
:1098EC000000000000000000F4020020F402002040
:1098FC0012010002EF020140E32F000107030102F5
:10990C00030109020000000100C032080B00020232
:10991C0002000009040000010202000005240010EE
:10992C00010524010201042402020524060001079A
:10993C0005800310000A09040100020A0000000758
:10994C0005800240000007050002400000040309E6
:10995C00040E035A455048595200000000000010F4
:10996C00035553422D4445560000000000000022D0
:10997C00033031323334353637383941424344457C
:10998C004600000000000000000000000000000085
:03999C00000000C8
:1099A000000000001F0300201B7F0000ED170000D7
:1099B000C1140000000000000000000003000000CF
:0899C000F400002015E015E0A1
:00000001FF
